:1000000058050020D10E000073280000490E0000A2
:10001000490E0000490E0000490E0000490E000084
:10002000490E0000490E0000490E0000410D00007D
:10003000490E0000490E0000ED0C000009280000E8
:10004000910E0000910E0000910E0000910E000034
:10005000910E0000910E0000910E0000910E000024
:10006000910E0000910E0000910E0000910E000014
:10007000910E0000910E0000910E0000910E000004
:10008000910E0000910E0000910E0000910E0000F4
:10009000910E0000910E0000910E0000910E0000E4
:1000A000910E0000910E0000910E0000910E0000D4
:1000B000910E0000910E0000910E0000910E0000C4
:1000C000910E0000910E0000910E0000910E0000B4
:1000D000910E0000910E0000910E0000910E0000A4
:1000E000910E0000910E0000910E0000910E000094
:1000F000910E0000910E0000910E0000910E000084
:10010000910E0000910E0000910E0000910E000073
:10011000910E0000910E0000910E0000910E000063
:10012000910E0000910E0000910E0000910E000053
:10013000910E0000910E0000910E0000910E000043
:10014000910E0000910E0000910E0000910E000033
:10015000910E000000000000000000000000000000
:10016000000000000000000000000000000000008F
:10017000000000000000000000000000000000007F
:10018000000000000000000000000000000000006F
:10019000000000000000000000000000000000005F
:1001A000000000000000000000000000000000004F
:1001B000000000000000000000000000000000003F
:1001C000000000000000000000000000000000002F
:1001D000000000000000000000000000000000001F
:1001E000000000000000000000000000000000000F
:1001F00000000000000000000000000000000000FF
:10020000DEE61E284CBBCE8F023500003C0000000D
:10021000008000000100000000000000000000005D
:10022000FFFF02910000000000000000000000003D
:1002300000000000000000000000000053B94AB9AF
:10024000002908BF00281CBF4FF0FF314FF0FF30DE
:1002500000F07CB9ADF1080C6DE904CE00F006F8B1
:10026000DDF804E0DDE9022304B070472DE9F04732
:100270008C46089D04468A46002B4AD18A4217467E
:1002800062D9B2FA82F64EB1C6F1200E01FA06F337
:10029000B740B44020FA0EFE4EEA030A4FEA174870
:1002A000230C1FFA87F9BAFBF8FE08FB1EAA0EFB07
:1002B00009F243EA0A439A420BD9FB180EF1FF31C7
:1002C0002CBF012000209A4202D9002800F02A8188
:1002D0008E469A1AA3B2B2FBF8F008FB102200FB7C
:1002E00009F943EA0244A14507D93C1900F1FF335B
:1002F00002D2A14500F210811846A4EB090440EA9D
:100300000E4000211DB1F4400023C5E90043BDE8C3
:10031000F0878B4208D9002D00F0F2800021C5E95A
:10032000000C0846BDE8F087B3FA83F100294ED1EE
:100330006345C0F0E880824240F2E5800846002D27
:10034000E5D0C5E9004AE2E702B9FFDEB2FA82F67B
:10035000002E40F099808B1A4FEA124E1FFA82F855
:1003600001214FEA144CB3FBFEF20EFB123008FBE6
:1003700002F94CEA004CE14508D917EB0C0C02F1EC
:10038000FF3302D2E14500F2CA801A46ACEB090CF9
:10039000A3B2BCFBFEF00EFB10CC08FB00F843EA56
:1003A0000C44A0450ED93C1900F1FF332CBF4FF08F
:1003B000010C4FF0000CA04503D9BCF1000F00F078
:1003C000A8801846A4EB080440EA02409AE7C1F16D
:1003D00020048B4002FA01FE0CFA01F6E24020FAFA
:1003E00004F72CFA04FC00FA01F813433E431F0CF7
:1003F000320C1FFA83F9BCFBF7F007FB10CC00FBB3
:1004000009FA42EA0C4CE24508D913EB0C0C00F156
:10041000FF3202D2E24500F289801046ACEB0A0CB2
:10042000B6B2BCFBF7FA07FB1ACC0AFB09F946EA9D
:100430000C42914506D99A180AF1FF3601D291452E
:100440007AD8B2464AEA0040A2EB0902A0FB0E6746
:10045000BA42B446B94602D307D1B04505D2B6EB8D
:100460000E0C67EB030301389946002D6BD0B8EBF7
:100470000C0362EB090202FA04F4CB40CA400021EB
:100480001C43C5E9004242E7B740C6F1200201FA29
:1004900006F3B44021FA02FC4FEA174E20FA02F2AA
:1004A0001FFA87F8BCFBFEF11A430EFB11CC01FBCF
:1004B00008F0130C43EA0C4C604507D917EB0C0C01
:1004C00001F1FF3301D2604533D81946ACEB000C83
:1004D00092B2BCFBFEF00EFB10CC00FB08F342EA2C
:1004E0000C4C634507D917EB0C0C00F1FF3201D21D
:1004F000634525D81046ACEB030340EA014130E7E1
:100500002946284603E7841A6CEB030301209A4628
:1005100015E702383C4455E702383C44EDE6023A20
:10052000BC4433E7AEF1020E3B44D2E602389C44B1
:1005300074E70239BC44C9E7AAF1020A1A4481E708
:100540000238BC44D7E72946E1E600BF704700BF48
:100550002DE9E04F2746A046A146A246A346A44661
:10056000A2B02DEC000A84F3008825462646A44755
:100570003DEC000A22B0BDE8E08F00000B680133BB
:100580000B60014B1B681847980E00202DE9F04FB7
:1005900085B00E9C9B46012CB8BF0124012B0CBFDB
:1005A0003023202316468246884601250A2700224A
:1005B000DFF86C900293B6FBF9F301930AB9B145E9
:1005C0001CD8019B414603F13000D0470122013580
:1005D000019B013F09FB13660A23012FB9FBF3F9C5
:1005E000E9D1414606F13000D047BBF1030F02D1FB
:1005F000641B002C0EDC05B0BDE8F08FBC42E7DBCD
:10060000BBF1020FE4D84146029803920135D0476E
:10061000039ADDE741462020D047013CE9E700BFCF
:1006200000CA9A3B014B1860704700BF980E00202B
:10063000002313B502AC44F8043D02460B460348C0
:10064000214601F058FE02B010BD00BF7D0500003C
:100650004FF02003EFF3118183F31188BFF36F8F05
:100660000123094AC2F8003502F55B521032536388
:100670001360C2F83432C2F8303481F31188BFF30A
:100680006F8F0020704700BF001000500A2838B557
:100690000446074D04D1286843680D215B689847DC
:1006A00028684368E1B25B689847204638BD00BFC0
:1006B0000800002010B5044C204600F069FF2046D9
:1006C000BDE81040FFF7AEBF8D06000008B5044836
:1006D00001F06EF9034B1860FFF7ECFF002008BD36
:1006E000E43000000800002008B5114B1A686AB118
:1006F0004FF05022D2F80423D10707D500220D482D
:100700001A608368597A09B901F0CEFF0A4B1A685A
:100710006AB14FF05022D2F80423920707D5002285
:1007200001211A600348BDE8084001F0BDBF08BDC3
:1007300000510050DC0E00200451005000220D4BEF
:10074000C3F840214FF02002EFF3118182F31188AA
:10075000BFF36F8F084AD3F804051368C01A20F05E
:100760007F400344136081F31188BFF36F8F01F062
:10077000F5BC00BF005001502400002070B51548A2
:1007800001F016F910B3436801211B689847002453
:1007900001264FF480334FF400120F4D3146C5F857
:1007A0000845C5F84065C5F804330C4B15201C609E
:1007B0000B4BC3F88021224600F0E2FA152000F02E
:1007C000CFFA2046074B1E602E6070BD4FF0FF3001
:1007D000FBE700BFB932000000500150405101500A
:1007E00000E100E00850015070B5264EB0F1FF3F27
:1007F00008BF30464FF02003EFF3118483F31188D4
:10080000BFF36F8F204BD3F80455204B1B68EA1AB7
:1008100022F07F42B2F5000F1AD2411E21EAE171A7
:10082000B142A8BF3146501C0844B04294BF1818CA
:100830009819451B25F07F45134A20F07F43022D70
:10084000C2F8403506D984F31188BFF36F8F70BDAD
:100850000021E8E7D2F804350D49C31A23F07F439D
:100860005D1E8D4205D94FF400120A4BC3F80021DA
:10087000E9E7012B02BF023020F07F40C2F84005BB
:10088000E1E700BFFEFFFF00005001502400002000
:10089000FEFF7F0000E100E04FF02002EFF3118344
:1008A00082F31188BFF36F8F064AD2F80405064A17
:1008B0001268801A20F07F4083F31188BFF36F8F96
:1008C000704700BF005001502400002008B543B21B
:1008D000002B0CDB012200F01F018A405B0910494C
:1008E000203341F82320BFF34F8FBFF36F8F830076
:1008F00003F1A04303F540532F28D3F8002806D076
:10090000002A07DA02F00302023A012A02D8054A55
:10091000C3F80028002101F07DFF002008BD00BFC2
:1009200000E100E00001008030B54FF4004448F2DF
:10093000040585B04FF400411C4801F052FE2168C7
:100940001B4801F04EFE29681A4801F04AFE1022A9
:100950000021684602F011F823686846009302946B
:1009600000F0A0FD012000F0CDFD002000F0B6FD5C
:10097000002000F0DBFD0121002000F0F5FD00F07B
:10098000E9FD2C680C4801F02CFE0820FFF79EFFC3
:1009900024F00104BFF34F8FBFF36F8F640864002E
:1009A0002046214622462346FFF7D2FD3932000079
:1009B0005032000065320000833200002DE9F84318
:1009C0006E4801F00EFE0021DFF8FC816C4F6D4D8A
:1009D00058F82140CA0301F5C07347F823406A481C
:1009E00002F500434E1C01F0FCFD684B14F0100FA3
:1009F0006749684808BF194601F0F3FD14F0040F79
:100A000014BF72212D21284601F0EBFD14F0020FD6
:100A100014BF77212D21284601F0E3FD14F0010FCA
:100A200014BF78212D21284601F0DBFD14F4807FCE
:100A300014BF6C212D21284601F0D3FD564801F04A
:100A4000D0FD202E3146C3D1544B4D4AC3F3C5319E
:100A5000C3F30E03C3F50043C3F34313C2F80015F9
:100A6000C2F80435D2F80015D2F804254C485201DA
:100A700001F0B7FD484801F0B4FD01F0C7FE0146A2
:100A800010B1484801F0ADFD434801F0AAFD4648C9
:100A900001F0A7FD0021DFF83481394F394D58F8B6
:100AA00021404A0301F5E07347F823403F4802F52F
:100AB00000534E1C01F095FD344B14F0100F3449D7
:100AC000344808BF194601F08CFD14F0040F14BF20
:100AD00072212D21284601F084FD14F0020F14BF6D
:100AE00077212D21284601F07CFD14F0010F14BF61
:100AF00078212D21284601F074FD14F4807F14BF65
:100B00006C212D21284601F06CFD234801F069FD80
:100B1000202E3146C3D10024194D1F4801F061FD3C
:100B2000C5F88044224801F05CFDDFF8A480C5F8D8
:100B3000C044DFF8A0901F4D05EBC406777955F847
:100B40003420002F14BF43464B4621461A4801F07B
:100B500048FD57B91948013401F043FD192CEBD178
:100B60000D48BDE8F84301F03CBD3079FFF7AEFE1B
:100B700008B11348EFE71348EDE700BF1531000057
:100B8000003000504D31000038310000FE300000D0
:100B9000F5300000223200000B340000E07F00003E
:100BA0005031000096310000C6310000E8310000ED
:100BB000FC3100002C2F000018320000253200000C
:100BC0002C32000034320000AC2E0000F42F000064
:100BD0000A3100000231000010B5F0B1EAB1104B4B
:100BE000994210D9541803F61D239C420ED801F0E7
:100BF00097FE0020BDE81040714672467346F446E9
:100C00008EF3008C7447074B994203D9064B541856
:100C10009C42ECD94FF0FF30ECE76FF01500E9E7AC
:100C20000302FF002F01FF003801FF002DE9F04F04
:100C3000824685B0894621B30026DFF858B0DFF838
:100C4000588001AF5BF8264098E80700544487E8D5
:100C500007000C223946204601F052FE054600B935
:100C600094B90136052EEDD16FF00D05284605B07B
:100C7000BDE8F04F714672467346F4468EF3008C21
:100C800074476FF01505F1E73C222146484601F014
:100C900047FEEBE7743000005C2E000004488168DA
:100CA000406A884203D003494FF080520A6070477F
:100CB0001401002004ED00E0094A0A49936809681C
:100CC0005866996608494B6843F080534B6000238F
:100CD00083F31188BFF36F8F9368986E704700BFDE
:100CE00014010020E030000000ED00E012498A68A5
:100CF0004FF028001044EFF3098C80E8F01F20200B
:100D000080F31188BFF36F8F0C4F4FF000664A6A73
:100D10008A603E60506E0023536680F3118804B5EC
:100D2000104601F0ADFDBDE8044002F1280090E856
:100D3000F01F8CF3098870471401002004ED00E0D7
:100D40001EF0040F0CBFEFF30880EFF309808169F8
:100D500011F8021C0229FFD001B501F086FD01BD8A
:100D600043B2002B08DB012200F01F0002FA00F062
:100D7000024A5B0942F82300704700BF00E100E02F
:100D800043B2002B01F10101A8BF03F160434FEA18
:100D90004111B8BF054BC9B2ABBF03F5614300F0C9
:100DA0000F0083F800131954704700BF14ED00E0E2
:100DB00073B51E460A9B05460093099B8C1801F0EB
:100DC000AFFE0B4AA4F1200323F0070322F0010237
:100DD0009A61069A1E605A60079A9A60089ADA60C9
:100DE0004FF08072DA61AB6400236B6602B070BDB5
:100DF000FD250000F8B505460C4617461E4600F0D6
:100E0000C1F90A4B3C4428469D6024F0070401F0D8
:100E100037FD304684F30988002163B681F31188D9
:100E2000BFF36F8F0022002301F0E8FB14010020C4
:100E3000014910220A60704710ED00E0404080F345
:100E4000118830BF704700BFEFF30880EFF30981CE
:100E5000724601B500F0BEF801BD00BF30BFFFF71C
:100E6000FDBF00BF08B5084B084A23F07F0393601D
:100E7000BFF34F8FBFF36F8F00F0DAFD00F0E2FD9C
:100E800000F04EF900F01CFE0000000000ED00E054
:100E900001B572B60B4A106A00281EBF002111620C
:100EA00001F0DBFD62B6EFF30580A0F110004FEA20
:100EB000C0000549014409C99847BDE801400349FC
:100EC0000847000014010020C82B00009D0C000002
:100ED00001F09FFB202080F3118808484FF4006147
:100EE000401880F30988EFF314800221084380F34F
:100EF0001488BFF36F8FFFF7B5FF0000980600203E
:100F00000C4B9A6A9A6A9A6A920708D55A6B9A6A3F
:100F1000120604D518B19A6A22F080029A62002063
:100F20009A6A9A6A9A6A9A6A42F0FF029A6208700A
:100F3000704700BF00ED00E00D4B9A6A9A6A9A6A0A
:100F4000920508D59A6B9A6A120404D518B19A6A68
:100F500022F400429A6200209A6A9A6AD205044AF0
:100F600058BF9B6A936A43F47F439362087070474B
:100F700000ED00E0074B00209A6A9A6A9A6A9A6A22
:100F80009A6A9A6A9A6A9A6A6FEA02426FEA124207
:100F90009A62704700ED00E00D4B9A695A695A69F0
:100FA000D0070FD45A6991070CD45A69520709D453
:100FB0005A69100706D45A69D10603D45A699206B1
:100FC00058BF5A695A6942F0FF025A61704700BF20
:100FD000D0ED00E0F0B5414B8BB05B680025C3F36A
:100FE000080385F31188BFF36F8F02F07F44B4F1DB
:100FF0007F4F1FD112F001041BD0560602F00804E7
:1010000068D482F00402C2F3800564B1EFF38986EC
:101010000022033B8DF80720042B4CD8DFE803F0B7
:101020000C4D51424900EFF38886F1E70646012551
:10103000EEE725462E46EBE7284BDA6A92073AD4CC
:10104000DC6A14F0804408D028331B78EBB101200F
:101050000DF10701FFF754FF04469DF8073093B9DF
:101060002022314602A801F05BFC099B6DB3C3F35B
:10107000080222B96FEA53236FEA4323099302A9B6
:10108000204601F0F0FB0BB0F0BD154B1B782BB1E7
:1010900001200DF10701FFF74FFFDDE7114B1C8821
:1010A000A7B217B1FFF766FFD6E70F4B5C69002CBC
:1010B000D3D0FFF771FF0024CFE70DF10701002027
:1010C000C8E70DF107010020E5E723F4FF7323F0E3
:1010D0000103D3E7002CA9D00E4699E700ED00E00C
:1010E00029ED00E02AED00E0D0ED00E0024A53696E
:1010F00043F010035361704700ED00E0BFF34F8FE2
:101100000549064BCA6802F4E0621343CB60BFF3A3
:101110004F8F00BFFDE700BF00ED00E00400FA05BF
:10112000002320210348C2180133452B82F8001305
:10113000F9D1704700E100E038B505464FF02003D3
:10114000EFF3118483F31188BFF36F8F00F098FEE3
:101150000A4B9B68AB420BD1094B5A68C2F3080299
:1011600012B92046FFF7A8FD5A6842F080525A6033
:101170002046BDE8384001F086BC00BF14010020C5
:1011800000ED00E010B50E4B88B002930D4B0E4CF5
:1011900003930E4B08A8049302AB40F81C3D0C4A85
:1011A0002346012100F002F900230793094B012196
:1011B000E41A05A80593069400F002F908B010BDE2
:1011C00000000020000000000000012006000100D7
:1011D000000000200000002010B50B680C7A23F0FE
:1011E0001F0304F01F021A43CB68640923F01F0396
:1011F000044943F0010343EA44038860CA600B6179
:1012000010BD00BF90ED00E02DE9F04F804689460B
:1012100014460027484D85B04F4507DA58F8273067
:101220005E68C6B31F2E05D86FF01504204605B0C2
:10123000BDE8F08FF206F7D1D3F800A01AF01F0F27
:10124000F2D1504601F046FB834606EB0A00013816
:1012500001F040FB8345E7D11BF1160FE4D0631E7C
:101260005B45E1DBC5F808B0E86858F82710C5F819
:1012700008B02E6920F01F00D1E900321A449842CC
:1012800046F01F0602F1FF3A18D1564505D15FFA24
:101290008BF001F0FDFA0137BEE7C5F808B0EB6846
:1012A00022F01F0203F01F031A43EA60E0B201F0CC
:1012B000EFFA10F1160FB7D0441CECE7C5F808B0F0
:1012C0002A69013B23F01F0302F01F021343564516
:1012D000E0B22B61EBD001F0DBFA10F1160FA3D0D6
:1012E000C5F808B0EA689DF80830013E62F30403CF
:1012F0008DF808302B699DF808205B0863F34712CE
:101300008DF8082058F827200130D2E90032134424
:10131000009323F01F031E44A6EB0A06C4B226F076
:101320001F060F2C03963FF67FAF20466946FFF756
:1013300053FF0134AFE700BF90ED00E00522034BFF
:101340005A60BFF34F8FBFF36F8F704790ED00E08F
:10135000BFF35F8F0022014B5A60704790ED00E0B1
:1013600070B50E4D2E68102E15D80024FFF7F0FF33
:101370000B4B0C4A1A63A64205D10B4B1E70FFF7AC
:10138000DDFF002070BD6968204601EB0411FFF706
:1013900023FF0134EFE74FF0FF30F3E78830000020
:1013A00090ED00E0AAFF44005401002010B5034C6A
:1013B0002278FFF729FF207010BD00BF54010020E4
:1013C0002DE9F74F894607460026DFF89080DFF8C1
:1013D00090A0214C4E4519DAD7F804B0BBF1000FAC
:1013E00036D03B681846019301F074FA019B05461C
:1013F0000BEB0300013801F06DFA1423854203FB67
:1014000006F306D06FF0150248F8032003B0BDE8DC
:10141000F08F15F1160F48F80350F7D09AF8002016
:10142000AA42F3DDA5604344A560E068197B60F340
:10143000040119732169187B490861F34710187377
:10144000E26822F01F025A60226922F01F021A612C
:1014500001360C37BEE700BF90ED00E02800002009
:101460005401002070B50C4B0E461C7805462346EF
:1014700000210A4A0F2B0BDD094B191D1868FFF7D5
:10148000ABFE224631462846BDE87040FFF7BCBEA1
:10149000936011610133EDE75401002090ED00E00D
:1014A0002800002082680C4B9A60036883F38888C8
:1014B000436883F38988027B02F00101EFF3948390
:1014C00023F00303920748BF43F0020309B143F03E
:1014D000010383F39488704700ED02E0084AD36863
:1014E00048B123F400531B041B0C43F0BF6343F4C7
:1014F0000033D36070479BB243F40053F5E700BF5D
:1015000000ED00E0084AD36840B19BB243F4804349
:1015100043F0BF6343F40033D360704723F4804348
:101520001B041B0CF4E700BF00ED00E0084AD36881
:1015300040B19BB243F0080343F0BF6343F4003370
:10154000D360704723F008031B041B0CF4E700BFB3
:1015500000ED00E0034AD2F88C3043F44063C2F857
:101560008C30704700ED00E0084B1A6818B142F06B
:1015700001021A60704722F001021A601A6811B164
:1015800042F00202F5E722F00202F2E7D0ED00E0BD
:10159000014B1860704700BF9C0E00204FF0805236
:1015A000094B0020C3F86422C3F86822C3F828223C
:1015B000C3F830221022054BC3F840244FF05023CB
:1015C000C3F81406704700BF002584500030005057
:1015D000F0B54B79012B2DD0032B28D110248B791A
:1015E000032B24D1CE792EB1012E20D103689B6824
:1015F0001B79E3B10B79012B1ED020D3022B16D11E
:1016000000220E2547F6122C03689B681F680B68A2
:10161000634578D030D8B3F5965F6ED01BD8B3F55C
:10162000167F58D00ED8B3F5967F00F081806FF00A
:1016300022005EE00024D2E74FF48072E1E700224E
:101640001546DFE7B3F5966F54D0B3F5166FEED1BC
:101650004FF41D2341E0B3F5615F50D004D8B3F5DA
:10166000165FE4D1344B38E0B3F5964F49D0B3F56B
:10167000E14FDCD1314B30E0B3F5E13F4CD012D833
:101680004DF6C02C634541D005D8B3F5164FCED1E9
:101690004FF41D0321E0B3F5614F3AD0B3F5963F07
:1016A000C5D1274B19E0B3F5E12F3BD009D8B3F5ED
:1016B000613F34D0DFF898C06345B8D14FF0806304
:1016C0000BE0B3F5612F30D0DFF888C06345AED1B1
:1016D0004FF0805301E04FF41C33C7F824353243F8
:1016E00083682C43224303C9C7F86C2583E80300B1
:1016F0000020F0BD4FF49E23EFE7124BEDE7124BB5
:10170000EBE7124BE9E74FF40003E6E74FF465031C
:10171000E3E74FF46B03E0E74FF0EB73DDE74FF0E7
:101720006C73DAE74FF0E863D7E74FF07063D4E704
:101730004FF4A033D1E700BF0050270000C0750070
:1017400000903A0100B0130000F03A0000A04E00F3
:1017500090D0030040420F00026870B59268184BA9
:1017600014684FF48012856803219A6014260022C1
:10177000C3F85012C3F85822C4F80C651626C4F8F2
:1017800014654FF400269E60C3F84C12C3F854222F
:101790001323C4F8083515232946C4F81035FFF77C
:1017A00017FF58B90823C4F800351D440123C4F8B5
:1017B0001001C4F83455C4F83835236070BD00BF3B
:1017C000002584502DE9F0430025214C214E54F88A
:1017D000048CDFF8889085B0A84503D8002005B0B8
:1017E000BDE8F083636A96E807001F6801AB83E8F1
:1017F00007000C221946384601F082F890B98FB1E3
:10180000636A21691B681A6991420BD19A69A169BF
:10181000914207D8E169914204D962695B6932EA71
:1018200003030AD0276A67B10B4800F0DAFE404094
:1018300080F311884FF0040002DFE36801351C4497
:10184000CAE7484600F0CDFE636A1F60F5E700BFB7
:101850003C020000682E0000B1330000DA330000C3
:10186000054B1868043B1B68072B03D1831E5842A5
:1018700058417047002070473401FF004FF050235B
:10188000D3F85825034B02F00102D340024A1360FB
:10189000704700BF0020A107AC0E0020314A08B5F8
:1018A000136843F0020313600022D30003F57F03A3
:1018B000D3F80013013107D0D3F800130132D3F865
:1018C0000433202A0B60F0D1FFF7CAFF002842D171
:1018D000FFF7C6FF38B1244B244A1A604FF050235B
:1018E0000122C3F85825FFF7BBFF10B10022204B9F
:1018F0001A60FFF7B5FF50B14FF05023D3F8002422
:10190000D10742BF0022C3F81421C3F81821194B94
:101910001B68072B0ED1184B1B68023B012B09D803
:101920004FF05023D3F80024D20744BF6FF00102D8
:10193000C3F80024FFF794FF10B165220F4B1A6023
:101940000F4AD2F88C3043F44063C2F88C30BDE8C3
:101950000840FFF793BF2922084B1A6003221A633D
:10196000B6E700BFD0ED00E0309503504400EFBE75
:101970004C2503503001FF003401FF000C4700509C
:1019800000ED00E070B50026084B53F82040013010
:1019900053F82050A54200D870BD236820465B68EC
:1019A000984700B166600C34F4E700BFCC3000000B
:1019B000104B70B505461E460F4C9C4204D10E4C90
:1019C000B44209D1002412E062681AB12268126898
:1019D000AA420CD00C34F0E763680BB90C34EFE783
:1019E00023682846196800F07EFF0028F6D12046BB
:1019F00070BD00BF240F0020B80E002008B50B4DAD
:101A00004FF02002EFF3118382F31188BFF36F8F41
:101A100001F0ABF8012104460228D8BF084601F0C6
:101A2000B4F82C62FFF70AFAEAE700BF14010020BD
:101A30000248034A0021121A00F09FBF0000002054
:101A40005801002008B50648064A0749121A00F056
:101A500067FFBDE80840054A0549064800F060BF39
:101A6000980E0020380F00206034000000000000B5
:101A70006034000000000020012208B50B4B02205A
:101A80001A70FFF77FFF0A4A0A490B4800F0A9FDC8
:101A90000320FFF777FF00F087FA00F0C9FB074A41
:101AA000137B23F00103137308BD00BF5501002011
:101AB000FD3000000D3400002A340000A800002092
:101AC00080B5374BA2B083F308880025E023354C5E
:101AD000012784F82230E57725766576A576E576C8
:101AE000636A314E43F4E0236362636A43F4002384
:101AF0006362A563FFF7FAFAFFF79AF94FF0FF3335
:101B0000A362E36207AB6C222946184600F035FF5A
:101B1000264C8DF82970A0602846FFF733FF384621
:101B2000FFF730FF00F0F0F9214B66624FF480625E
:101B3000CDE90473CDE902551E4BCDE900551E4990
:101B4000304600F017FA737B23F0040213F01B0FEA
:101B5000727304D1B36913B9304600F0DFF8174B44
:101B6000012205930F23CDE903320023144DCDE963
:101B7000013300934FF4A072124B1349284600F032
:101B8000F9F96B7BE56023F004036B730F4B4FF4A3
:101B90008062C4E906330849064B0348FFF72AF977
:101BA000980E002000ED00E0A800002014010020A5
:101BB00051340000791A000058010020563400000A
:101BC0003C000020FD190000580500202C010020D9
:101BD00010B5084C23685BB1FEF75EFE2368064A29
:101BE000184410610021BDE81040184600F0CDBF38
:101BF00010BD00BF4C01002014010020F8B50D46B7
:101C00004FF02003EFF3118483F31188BFF36F8F3C
:101C10004FF4004140F2E73600270022E1FB006765
:101C2000094B30461A6139464FF47A720023FEF7A9
:101C300005FB064B1860064B1D60FFF7C9FF84F3D8
:101C40001188BFF36F8FF8BD140100204C010020F4
:101C5000480100204FF02003EFF3118183F3118836
:101C6000BFF36F8F044B9A68D37B013BD37381F32F
:101C70001188BFF36F8F704714010020094B03F1E7
:101C80002802824205D19B688B4202D14B7BDB0646
:101C900007D1D1E900231A600A6853600023C1E923
:101CA000003370471401002038B50D4C024604F192
:101CB000280000F0FEFE054600B9E568A3684AB9B1
:101CC0005A7BD20606D1AA6922B9DA897F2A01D9BC
:101CD000636238BD9D4201D0FFF77AFF6562F8E785
:101CE0001401002010B54FF02003EFF3118483F3AB
:101CF0001188BFF36F8F084B00209A68D37B0133A4
:101D0000D373FFF7D1FF84F31188BFF36F8FBDE862
:101D1000104000F0C4BE00BF14010020F8B54FF021
:101D20002003EFF3118483F31188BFF36F8F164AFA
:101D3000114651F8283F8B420CD05BB1D66A90F91E
:101D40000E5093F90E70AF420BDCB34202D01B6809
:101D5000002BF6D1D36A01604360D36A1860D06269
:101D600005E05A68C0E900325A6810605860437B49
:101D700063F07F0343730020FFF796FF84F311881D
:101D8000BFF36F8FF8BD00BF14010020F8B5044603
:101D90004FF02003EFF3118583F31188BFF36F8FAA
:101DA00090F90D30002B03DA01461848FFF766FF63
:101DB000174A02F12801D2E90A308B420BD053B105
:101DC00094F90E6093F90E70B7420ADC834202D098
:101DD0001B68002BF6D1C4E90010D36A1C60D462E2
:101DE00005E05968C4E9003159680C605C60637BA8
:101DF000906863F07F036373031B58425841FFF7F9
:101E000053FF85F31188BFF36F8FF8BD3C010020AD
:101E100014010020154A164938B50C689368A3428E
:101E2000144603D1BDE83840FFF7D2BE00250D604F
:101E300010490968B9B1D9897F2914D80E4993F995
:101E40000E5009688D420EDB0C498B420BD099690C
:101E500049B91169814203DC1846FFF797FFE1E7B2
:101E6000091A116138BD00232361FBE7140100202A
:101E7000440100204C010020480100203C000020CB
:101E8000036D70B5044603B1984704F1180000F0E3
:101E900056FE4FF02003EFF3118583F31188BFF353
:101EA0006F8F204600F0DBFD0646D8B194F90D3067
:101EB000002B07DA21461248FFF7E0FE637B03F0B0
:101EC0007F0363730F4B9868021B50425041FFF72A
:101ED000EBFE637B43F00803637385F31188BFF364
:101EE0006F8F70BD637B9B07F3D52146A068FFF71A
:101EF000C5FE637BA66023F002036373E9E700BFBE
:101F00003C010020140100200021044B084603F18D
:101F10002802C3E90A22FFF771BE00BF14010020A6
:101F2000014B9868704700BF1401002010B54FF0B6
:101F30002002EFF3118482F31188BFF36F8F427B8D
:101F4000510704D484F31188BFF36F8F10BD22F0C2
:101F5000040112F01B0F417303D183690BB9FFF722
:101F6000DDFE2146BDE81040014800F081BD00BF04
:101F70005601002030B587B00E9D044604950D9D96
:101F800003950C9D02950B9D01950A9D0095FEF70A
:101F90000FFF044B9B6813B9236607B030BD1B6E5F
:101FA000FAE700BF140100202DE9F04F284E294D1B
:101FB000B04687B0B54205F1300410D3FFF74AFEB2
:101FC0004FF4004940F2E7360027224CDFF888A0A2
:101FD000444521D307B0BDE8F04FFFF783BE54F866
:101FE000043C059354F8103C049354F8143C0393B8
:101FF00054F8183C029354F81C3C019354F8203CCC
:10200000009354E90A2354E90C01FFF7B3FF54F895
:10201000303CDD642546CDE7616A4B1C04D0256861
:1020200021B92846FFF782FF3034D1E7B346BC46DA
:10203000E9FB01BC4FF47A72002358466146FEF773
:10204000FDF85146421C05F1180000F043F8EBE79B
:10205000240F0020240F0020BF2A0000034B1B6820
:102060000BB9FEF719BC0020704700BF50010020DB
:10207000036840B1084A5268904204D01BB19A6884
:1020800081680A449A604268136003685A600023BA
:10209000C0E90033704700BFB00E00200B4B10B5F5
:1020A0001C689C4208BF0024FFF7D8FF54B1A36806
:1020B000181A20EAE070064B1B6913B19842A8BFBA
:1020C000184610BD6FF00040F5E700BFB00E0020CD
:1020D0001401002070B504461646C1604FF020037D
:1020E000EFF3118583F31188BFF36F8FFFF7B6FF0E
:1020F000012EACBF80190130174BA0601A689A42BC
:1021000001D05E6832B95A68236062605A68146010
:102110005C600BE09068A168884216DD411A91600E
:102120005168C4E9002151680C6054601A689A42F1
:1021300006D0944204D1FFF7B1FF0021FEF754FB13
:1021400085F31188BFF36F8F70BD091A9642A160A5
:10215000D9D01268D6E700BFB00E00202DE9F04BB1
:102160000446FFF757FE4FF02003EFF3118583F38A
:102170001188BFF36F8F214F214EB846DFF884904E
:102180003460D9F8004032684C45D7E900BC05D02E
:1021900024B1A368934214DD9B1AA36000241BEBB7
:1021A00002004CEBE271C8E900013460FFF776FFF2
:1021B0002146FEF719FB85F31188BFF36F8FBDE849
:1021C000F08B1BEB03004CEBE371D31A336000235D
:1021D000C7E90001A3602046FFF74AFF85F3118895
:1021E000BFF36F8FE36898474FF02003EFF311853B
:1021F00083F31188BFF36F8FC3E700BF0000002097
:1022000050010020B00E002038B5074C074DAC42FD
:1022100001D3002038BD04F114032046C4E905337E
:1022200000F00DF81C34F2E7240F0020240F0020EA
:1022300008B5FEF7C3FBBDE80840FEF775BBFF23FA
:102240002DE9F74F4568002229464FF00C0A4FF060
:10225000200B0789046805FB07FCC372837A64447A
:102260000193019B934208DC002319468F4205EB42
:10227000030C21DC03B0BDE8F08FBCFBF1F3202B95
:1022800084BF1F3393FBFBF30AFB02FED0F80C80E4
:102290004FEA910108EB0E0606F10409C6E901991F
:1022A00021F0030194BFC27248F80E4002F101020E
:1022B00088BF04EB8304D4E7C268066802F1040E09
:1022C000F41846F803E093680131636093681C607A
:1022D00094606346CAE70020704770B50D46044617
:1022E0004520A04729465220A04729462346BDE85D
:1022F0007040522018472DE9F04F002705460E4642
:1023000092461C464FF0FF39B846BB4689B09AF852
:10231000000010B909B0BDE8F08FBBF1000F07D184
:10232000252800F04E813146A8470AF1010AEEE760
:10233000642868D01AD839280BD831285AD22D28C9
:1023400000F04681302846D0252808D13146A847DC
:102350007AE0582800F0B480632800F02C813146E0
:102360002520A84731469AF80000F0E7702800F0D1
:102370009D800DD8692846D06C2803D16C2F26D1BA
:102380004C27D2E76828EAD1682F20D14827CCE72C
:10239000752870D017D87328E1D1226804F1040B96
:1023A00011460C4614F8010B002840F0F980B8F1F2
:1023B000030F40F013818C1AA9EB0404002C00F3E6
:1023C000F5805C4640E078287AD07A28C7D1002F83
:1023D000C5D10746A9E7B9F1000F0EDAB8F1000F31
:1023E00000F0F980A0F13009B8F1000F08BF4FF0FC
:1023F00002089AE7B9F1000FF4DB0A2202FB09098F
:10240000A9F13009F0E77A2F03D1D4F800B00434F1
:102410001EE06C2FF9D04C2FF7D14FF0000C4FF08D
:10242000FF3B073424F0070303F10804D3E900233A
:1024300012F1004043F100018C4508BF834506D2EC
:1024400031462846FFF749FF4FF0000B6DE79346F2
:10245000BBF1000F06DA31462D20A847CBF1000B67
:1024600009F1FF3943465A46CDF8009031462846D7
:10247000FEF78CF8E8E77A2F02D12268043411E0E5
:102480006C2FFAD04C2FF8D100214FF0FF300734D9
:1024900024F0070303F10804D3E90023994208BF9D
:1024A0009042CDD3CDF800904346DFE7314630204F
:1024B000A84731467820A8474FF008094FF0010897
:1024C0009AF80020702A05D123680434049300236D
:1024D00002930CE06C2FF7D04C2FF5D1073424F089
:1024E0000702136802F10804049353680293002260
:1024F0001023039205924022043A02990498C2F1F3
:10250000200CA2F1200ED04001FA0CFC40EA0C0095
:1025100021FA0EFE40EA0E0010F00F0008D10599D6
:1025200001B942BB4FF0300C08E0CDF814B0E3E73E
:1025300009288CBF4FF0570C4FF0300C31466044E7
:10254000CDE90523A847039B01330393DDE9052368
:10255000002AEAD1B8F1030F7FF476AF039BC3EBF7
:10256000490BBBF1000F7FF76FAF31462020A84722
:102570000BF1FF3BF5E7591E9945069107DBB8F1D2
:10258000010F06D1314630200792A847079A069BD3
:10259000B2E7B8F1020FFAD1079231462020F4E7F2
:1025A00031460292A8472146029AFAE63146202097
:1025B000A847013C02E73146206804F1040BA84714
:1025C000FFE65F46D8464FF0FF394FF0010BACE60F
:1025D0004FF00308A9E64FF00108A6E65C468346E3
:1025E000A3E60FB407B504A951F8040B0191FEF757
:1025F0001FF803B05DF804EB04B07047044608B55B
:10260000084611461A46A047FFF78AFCFEF794FDDC
:102610007047FFF743B90C228368C9B202FB01314E
:102620004B7A23B9087AB0FA80F04009704702204B
:1026300070470268F8B59768CCB286684FF02003FF
:10264000EFF3118583F31188BFF36F8F0C22624380
:10265000B1180B7A1BB3013BDBB20B7213BBB35047
:102660003A444B605368B3B90C23012103FB047354
:10267000DA7A1B8902F150221160002203F1502303
:102680001A600C21002001FB0464607285F311883C
:10269000BFF36F8FF8BD98470028E5D1F1E76FF0E1
:1026A0004400F3E70020F1E738B50C2483680546C1
:1026B00004FB0134012363724FF02003EFF3118117
:1026C00083F31188BFF36F8F23682BB160681A689A
:1026D0008342226008BF626081F31188BFF36F8F6D
:1026E00003B938BDD3E9012128469047E4E70368E0
:1026F0002DE9F041D0F808C005469F68CEB24AB136
:102700000C2373435CF803309A425CD013B11B680E
:10271000002BF9D14FF02003EFF3118083F31188E0
:10272000BFF36F8F0C2171430CEB01031C7A013452
:10273000E4B21C7280F31188BFF36F8F32B34FF095
:1027400050204FF0030EC0F808E3587AA0B94FF0BC
:10275000200EEFF311888EF31188BFF36F8F106096
:10276000D3F804E0BEF1000F20D15A604CF80120EC
:1027700088F31188BFF36F8F4FF050230321C3F804
:10278000041318B1D2E9013128469847012C0BD126
:102790000C237343FB586BB90C23012203FB067611
:1027A000B37A03F150231A6000200EE0CEF8002027
:1027B0005A60DDE7284698470028EDD13146284683
:1027C000FFF772FFF0E76FF00F00BDE8F081002225
:1027D000FFF78DBF10B50022044601210520FEF74A
:1027E000CFFA0520FEF7BCFA4FF050230222C3F8BF
:1027F000182503220020C3F80423A368C3E90000BE
:10280000A368C3E9030010BD7047704700207047FC
:10281000FEF71ABB43B2A9B1002B12DB01215B0901
:102820009B0003F1604303F56143D3F8802200F07D
:102830001F0001FA00F022EA0000C3F88002D3F87A
:1028400080327047002BFCDB01225B099B0003F107
:10285000604303F56143D3F8801200F01F0002FAD1
:1028600000F00843E9E700F0E9B80146006800F02D
:10287000E5B808B5FEF7F2FABDE80840FEF70EBA73
:1028800007B5002101A8FEF7EDFD03B05DF804FBDC
:1028900030B585B09DF808200D890B684C684989D2
:1028A00065F3040261F3471200938DF8082023F0CA
:1028B0001F03621E134423F01F030F2803930446D3
:1028C00005D86946FEF788FC204605B030BD6FF09C
:1028D0001504F9E740E800F313F4803FD8B208BFCD
:1028E0006FF0150070470138013910F8013F11F8F9
:1028F000012F934202D1002BF7D11A46981A704744
:1029000010B55AB10139841810F8012B11F8013FA4
:10291000A04201D09A42F7D0D01A10BD1046FCE771
:10292000F0B581EA0004A50703460BD0013B0A4439
:1029300091421DD1F0BD002AFCD011F8014B013AA3
:1029400003F8014B9C07F6D10C461D1F8F183E1B48
:10295000032E08D86FF00305940805FB0422A40099
:1029600023442144E2E754F8046B45F8046FEEE792
:1029700011F8014B03F8014FDAE70346F0B5C9B28D
:102980009C070FD11D4641EA012444EA04449F18E4
:102990007E1B032E0CD8940803EB840413449C4242
:1029A00009D1F0BD002AFCD003F8011B013AE7E78A
:1029B00045F8044BECE704F8011BF0E74FF0FF305B
:1029C00070470B46826892E8030083E8030000200A
:1029D000704703689B681B68D3F88004C3F88004C1
:1029E0007047036882689B681B68D3F8100138B190
:1029F000127A00200A700122C3F810011A60704791
:102A00004FF0FF30704782B002AA02F8011D00218A
:102A100003689B681B68C3F82011C3F84425012292
:102A2000C3F848259A60D3F820110029FBD0DA605A
:102A300002B0704708B50020FEF760FB70B5054690
:102A40000E46FFF76DFA314604462846FFF7F2FFBF
:102A50002046BDE87040FEF76FBBFFF7D6BE437B54
:102A6000DB0603BF8069B0FA80F0400900207047A0
:102A700021B9EFF3058008B9FEF71EB981F311887B
:102A8000BFF36F8F7047034620B9EFF305820AB991
:102A9000FEF712B983F31188BFF36F8F70474FF0C1
:102AA0002003EFF3118083F31188BFF36F8FFFF7DB
:102AB000EABF0368984214BF18460020704750F8D8
:102AC000103C70B50446A0F11805CBB14FF02003BF
:102AD000EFF3118683F31188BFF36F8F294650F807
:102AE000100CFFF7CBF814F80B3C23F0020304F8AA
:102AF0000B3C86F31188BFF36F8F002344F8103C22
:102B000014F80B3C284623F0140304F80B3CFFF7A1
:102B1000A6FF20B12846BDE87040FFF7FFB870BDA2
:102B200010B5029C8373047300230424C37344739D
:102B3000C0E90633C0E91333C0E9161210BD10B561
:102B40004FF02002EFF3118482F31188BFF36F8FEF
:102B500003683BB1FFF78CFA002084F31188BFF3C0
:102B60006F8F10BD6FF01500F7E710B54FF0200321
:102B7000EFF3118483F31188BFF36F8FFFF78EFAA1
:102B800084F31188BFF36F8F10BD70B504460E46F5
:102B90004FF02003EFF3118583F31188BFF36F8F9C
:102BA000FFF77CFA012805DDA04203DD314620460F
:102BB000FDF71AFE85F31188BFF36F8F70BD704764
:102BC000ACD6FF7F010000000000000011280000CB
:102BD0000000000011280000000000001128000083
:102BE0000000000011280000000000001128000073
:102BF00000000000E90600000000000011280000AD
:102C00000000000011280000000000001128000052
:102C10000000000011280000000000001128000042
:102C20000000000011280000000000001128000032
:102C30000000000011280000000000001128000022
:102C40000000000011280000000000001128000012
:102C50000000000011280000000000001128000002
:102C600000000000112800000000000011280000F2
:102C7000000000003D0700000000000011280000D7
:102C800000000000112800000000000011280000D2
:102C900000000000112800000000000011280000C2
:102CA00000000000112800000000000011280000B2
:102CB00000000000112800000000000011280000A2
:102CC0000000000011280000000000001128000092
:102CD0000000000011280000000000001128000082
:102CE0000000000011280000000000001128000072
:102CF0000000000011280000000000001128000062
:102D00000000000011280000000000001128000051
:102D10000000000011280000000000001128000041
:102D20000000000011280000000000001128000031
:102D30000000000011280000000000001128000021
:102D40000000000011280000000000001128000011
:102D50000000000011280000000000001128000001
:102D600000000000112800000000000011280000F1
:102D700000000000112800000000000011280000E1
:102D800000000000112800000000000011280000D1
:102D900000000000112800000000000011280000C1
:102DA00000000000112800000000000011280000B1
:102DB00000000000112800000000000011280000A1
:102DC0000000000011280000000000001128000091
:102DD0000000000011280000000000001128000081
:102DE0000000000011280000000000001128000071
:102DF000FD3000005106000000000000FD30000022
:102E0000CD06000000000000B9320000D527000008
:102E1000942E0000EB3000007D0700000000000051
:102E2000FD3000006113000000000000FD300000D4
:102E30009D15000000000000E4300000591700005C
:102E4000C4300000FD300000C51700000000000085
:102E5000FD3000000922000000000000DEE61E2810
:102E60004CBBCE8F02350000DEE61E28EAAC45B82A
:102E700002350000DEE61E284CBBCE8F0235000076
:102E8000CF27000033260000EF26000000000000DE
:102E900017260000000000000000000000010004F0
:102EA00000000000000000000401080C17010000F1
:102EB00007010000070100000701000007010000F2
:102EC00007010000070100000701000007010000E2
:102ED00007010000070100000701000007010000D2
:102EE00007010000070100000701000007010000C2
:102EF00007010000070100000701000007010000B2
:102F000007010000070100000701000007010000A1
:102F10000701000007010000070100000701000091
:102F2000070100000701000007010000AE320000A9
:102F300042010000B532000005010000BF32000070
:102F400014010000C832000015010000D132000059
:102F500039010000DA32000009010000E53200000A
:102F60000B000000F03200000B010000FA320000FC
:102F70000C010000043300000F0100000F330000BB
:102F8000100100001A330000110100002533000079
:102F90000E0100002F330000210100003833000033
:102FA0002201000041330000230100004A330000E9
:102FB00024010000533300002A0100005B330000AD
:102FC0008101000063330000000100006B3300004A
:102FD0001C010000743300001D0100007D3300005F
:102FE00017010000873300002F0100009333000019
:102FF0000401000017010000170100001701000084
:103000001701000017010000170100001701000060
:103010001701000007010000070100000701000080
:103020000701000007010000070100000701000080
:103030000701000007010000070100000701000070
:103040000701000007010000070100000701000060
:103050000701000007010000070100000701000050
:103060000701000007010000070100000701000040
:103070000701000000000000000200000004000042
:103080000008000000100000020000009030000066
:1030900000000000A233000006000000E0FF0F0067
:1030A00000000020AA33000021000000E0FF002003
:1030B000E3290000072A0000D3290000D1150000F1
:1030C000C32900000080005001000000B80E00205D
:1030D000000F00200C0F0020240F0020240F0020E0
:1030E000F5FFFFFF554152545F30007379735F6302
:1030F0006C6F636B005365637572650909004E6FF1
:103100006E2D53656375726509004E6F6E2D5365A4
:103110006375726500466C61736820726567696FDC
:103120006E0909446F6D61696E09095065726D69B8
:103130007373696F6E730A002530327520307825FD
:103140003035782030782530357820090025630027
:103150004E6F6E2D7365637572652063616C6C6173
:10316000626C6520726567696F6E203020706C61DB
:1031700063656420696E20666C61736820726567A0
:10318000696F6E20256420776974682073697A6599
:103190002025642E0A00436F756C64206E6F7420C6
:1031A000696E697469616C697A65207365637572AB
:1031B0006520736572766963657320286572722075
:1031C0002564292E0A005352414D20726567696FAC
:1031D0006E0909446F6D61696E09095065726D6908
:1031E0007373696F6E730A0025303275203078254D
:1031F000303578203078253035780900506572698F
:1032000070686572616C0909446F6D61696E0909C6
:103210005374617475730A002530327520252D3280
:10322000317325730009534B49500A000945525226
:103230004F520A00094F4B0A0053504D3A204E534B
:1032400020696D61676520617420307825780A00F7
:1032500053504D3A204E53204D535020617420302E
:103260007825780A0053504D3A204E5320726573EA
:10327000657420766563746F7220617420307825E0
:10328000780A0053504D3A20707265706172652063
:10329000746F206A756D7020746F204E6F6E2D53A1
:1032A000656375726520696D6167652E0A004E520F
:1032B000465F5030004E52465F434C4F434B004EEA
:1032C00052465F52544330004E52465F525443318F
:1032D000004E52465F4E564D43004E52465F55419A
:1032E00052544531004E52465F55415254453200CA
:1032F0004E52465F5457494D32004E52465F53502E
:10330000494D33004E52465F54494D455230004EB0
:1033100052465F54494D455231004E52465F544922
:103320004D455232004E52465F5341414443004E98
:1033300052465F50574D30004E52465F50574D3108
:10334000004E52465F50574D32004E52465F505726
:103350004D33004E52465F495043004E52465F5631
:103360004D43004E52465F465055004E52465F4513
:10337000475531004E52465F45475532004E524642
:103380005F4450504943004E52465F4750494F54A6
:103390004531004E52465F524547554C41544F52BD
:1033A0005300464C4153485F30005352414D5F300B
:1033B000004552524F523A2043616E6E6F74206640
:1033C000756C66696C6C204558545F415049207299
:1033D0006571756573742E0D0A005741524E494E42
:1033E000473A204F7074696F6E616C204558545F86
:1033F0004150492072657175657374206E6F742039
:1034000066756C66696C6C65642E0D0A0076322EEA
:10341000312E39392D6E6373312D332D6737646446
:10342000616236363462303462002A2A2A20426FC2
:103430006F74696E67205A6570687972204F5320E7
:103440006275696C64202573202573202A2A2A0A54
:10345000006D61696E0069646C6500000000000029
:10346000D7220000BD29000000C2010000010300B6
:10347000000000000090D003B00E0020B00E00202D
:10348000F02D00000000000000000000502E0000A1
:103490000000000000000000202E000000000000DE
:1034A00000000000082E0000802E00000C0000200C
:1034B000382E0000B0300000A00E0020FC2D0000CF
:1034C0000000000000000000142E000000000000BA
:1034D000000000002C2E0000000000000000000092
:1034E000442E00000000000000000000240F002017
:1034F000240F002000000000000000000F0000006A
:1035000000000000000000000000000000000000BB
:1035100000000000000000000000000000000000AB
:10352000000000000000000000000000000000009B
:10353000000000000000000000000000000000008B
:107FE0007FE97FE9F8F7F8BD7FE97FE9F8F71EBE82
:107FF0000000000000000000000000000000000081
:10800000781C0120F1990000D5D10000B99700003B
:10801000B9970000B9970000B9970000B997000020
:10802000B9970000B9970000B99700008197000048
:10803000B9970000B99700002D9700000FD10000FC
:10804000D5970000D5970000D5970000D597000080
:10805000D5970000D5970000D5970000D597000070
:10806000D5970000D5970000D5970000D597000060
:10807000D5970000D5970000D5970000D597000050
:10808000D5970000D5970000D5970000D597000040
:10809000D5970000D5970000D5970000D597000030
:1080A000D5970000D5970000D5970000D597000020
:1080B000D5970000D5970000D5970000D597000010
:1080C000D5970000D5970000D5970000D597000000
:1080D000D5970000D5970000D5970000D5970000F0
:1080E000D5970000D5970000D5970000D5970000E0
:1080F000D5970000D5970000D5970000D5970000D0
:10810000D5970000D5970000D5970000D5970000BF
:10811000D5970000D5970000D5970000D5970000AF
:10812000D5970000D5970000D5970000D59700009F
:10813000D5970000D5970000D5970000D59700008F
:10814000D5970000D5970000D5970000D59700007F
:10815000D5970000000000000000000000000000B3
:10816000000000000000000000000000000000000F
:1081700000000000000000000000000000000000FF
:1081800000000000000000000000000000000000EF
:1081900000000000000000000000000000000000DF
:1081A00000000000000000000000000000000000CF
:1081B00000000000000000000000000000000000BF
:1081C00000000000000000000000000000000000AF
:1081D000000000000000000000000000000000009F
:1081E000000000000000000000000000000000008F
:1081F000000000000000000000000000000000007F
:10820000DEE61E284CBBCE8F023500003C0000008D
:1082100014670000010000000080000000800000E2
:10822000FFFF0291000000000000000000000000BD
:1082300000000000000000000000000053B94AB92F
:10824000002908BF00281CBF4FF0FF314FF0FF305E
:1082500000F07CB9ADF1080C6DE904CE00F006F831
:10826000DDF804E0DDE9022304B070472DE9F047B2
:108270008C46089D04468A46002B4AD18A421746FE
:1082800062D9B2FA82F64EB1C6F1200E01FA06F3B7
:10829000B740B44020FA0EFE4EEA030A4FEA1748F0
:1082A000230C1FFA87F9BAFBF8FE08FB1EAA0EFB87
:1082B00009F243EA0A439A420BD9FB180EF1FF3147
:1082C0002CBF012000209A4202D9002800F02A8108
:1082D0008E469A1AA3B2B2FBF8F008FB102200FBFC
:1082E00009F943EA0244A14507D93C1900F1FF33DB
:1082F00002D2A14500F210811846A4EB090440EA1D
:108300000E4000211DB1F4400023C5E90043BDE843
:10831000F0878B4208D9002D00F0F2800021C5E9DA
:10832000000C0846BDE8F087B3FA83F100294ED16E
:108330006345C0F0E880824240F2E5800846002DA7
:10834000E5D0C5E9004AE2E702B9FFDEB2FA82F6FB
:10835000002E40F099808B1A4FEA124E1FFA82F8D5
:1083600001214FEA144CB3FBFEF20EFB123008FB66
:1083700002F94CEA004CE14508D917EB0C0C02F16C
:10838000FF3302D2E14500F2CA801A46ACEB090C79
:10839000A3B2BCFBFEF00EFB10CC08FB00F843EAD6
:1083A0000C44A0450ED93C1900F1FF332CBF4FF00F
:1083B000010C4FF0000CA04503D9BCF1000F00F0F8
:1083C000A8801846A4EB080440EA02409AE7C1F1ED
:1083D00020048B4002FA01FE0CFA01F6E24020FA7A
:1083E00004F72CFA04FC00FA01F813433E431F0C77
:1083F000320C1FFA83F9BCFBF7F007FB10CC00FB33
:1084000009FA42EA0C4CE24508D913EB0C0C00F1D6
:10841000FF3202D2E24500F289801046ACEB0A0C32
:10842000B6B2BCFBF7FA07FB1ACC0AFB09F946EA1D
:108430000C42914506D99A180AF1FF3601D29145AE
:108440007AD8B2464AEA0040A2EB0902A0FB0E67C6
:10845000BA42B446B94602D307D1B04505D2B6EB0D
:108460000E0C67EB030301389946002D6BD0B8EB77
:108470000C0362EB090202FA04F4CB40CA4000216B
:108480001C43C5E9004242E7B740C6F1200201FAA9
:1084900006F3B44021FA02FC4FEA174E20FA02F22A
:1084A0001FFA87F8BCFBFEF11A430EFB11CC01FB4F
:1084B00008F0130C43EA0C4C604507D917EB0C0C81
:1084C00001F1FF3301D2604533D81946ACEB000C03
:1084D00092B2BCFBFEF00EFB10CC00FB08F342EAAC
:1084E0000C4C634507D917EB0C0C00F1FF3201D29D
:1084F000634525D81046ACEB030340EA014130E761
:108500002946284603E7841A6CEB030301209A46A8
:1085100015E702383C4455E702383C44EDE6023AA0
:10852000BC4433E7AEF1020E3B44D2E602389C4431
:1085300074E70239BC44C9E7AAF1020A1A4481E788
:108540000238BC44D7E72946E1E600BF704700BFC8
:108550000149024804F00FBA78DE000092DE000004
:108560002DE9F04F85B00E9C9B46012CB8BF01242D
:10857000012B0CBF30232023164682468846012556
:108580000A270022DFF86C900293B6FBF9F30193FF
:108590000AB9B1451CD8019B414603F13000D047D0
:1085A00001220135019B013F09FB13660A23012FBC
:1085B000B9FBF3F9E9D1414606F13000D047BBF1F0
:1085C000030F02D1641B002C0EDC05B0BDE8F08F58
:1085D000BC42E7DBBBF1020FE4D8414602980392AC
:1085E0000135D047039ADDE741462020D047013CC2
:1085F000E9E700BF00CA9A3B014B1860704700BF13
:10860000B847012030B5002585B0CDE90101044609
:1086100001A90548039504F038F8DDE902309842D5
:10862000B8BF255405B030BD65C6000048B1054B44
:108630001A68054BB2FBF3F2044B504343F00103BD
:1086400018477047D047012040420F0050DD00001E
:10865000014803F01FBD00BF7848012030B500225B
:1086600087B00D490D4805F09EF900240E230C4DEE
:10867000CDE90243CDE90444CDE90044094B4FF470
:1086800080620949284603F08DFD0849284605F017
:1086900032F9204607B030BD518600001C00012091
:1086A00064000120FD89000078140120A7DE00008D
:1086B00008B500F033FA094804F08EF94023482247
:1086C0000749084805F03DF8074B084A4FF40040B9
:1086D0001A60BDE8084000F067BC00BF140001202C
:1086E000B825012048000120BC47012017CA00001E
:1086F000F8B500250C4BD3E8EF7FC3E8E25F002A12
:10870000F9D10A4C0A4E361B3611B54200DBF8BDD2
:1087100063685B792BB12368DB6813B13946204667
:10872000984701351034F0E70C0001201CDD0000F3
:108730002CDD0000044BD3E8EF2F0132C3E8E12F1A
:108740000029F8D1704700BF0C000120044A054BF6
:108750009B1AB1EBD30F34BF52F8310000207047A1
:10876000DCDC00001CDD0000094B4268C31A1B1151
:10877000013310B5137101224368064C5A712278F7
:10878000196012B9044803F085FC0123237010BD61
:108790001CDD00004803012078480120F8B50F4B8C
:1087A000D3E8EF4F621CC3E8E12F0029F8D12CB9C0
:1087B0000B4D0C4E761B3611B44200DBF8BD270181
:1087C000EB191B7B43B1EB595B6903B1984704225A
:1087D0000021E819FFF7C8FF0134EDE71000012080
:1087E0001CDD00002CDD0000144B37B59842044618
:1087F00002D3134B98421BD3002201A9114802F067
:10880000E9FF0546B8B90122019BD3E8EF1FC3E891
:10881000E02F0028F9D1019821463F22043004F0CE
:108820001EFD7E23019C84F8433084F844500434B8
:10883000204603B030BD044CFAE700BF18DA000050
:108840001CE6000048000120AFDE000050B1064BDE
:10885000984206D303F5905398422CBF0020012084
:1088600070470020704700BFB82501202DE9F84F60
:10887000434B05461B7803B940B34FF02003EFF399
:10888000118683F31188BFF36F8F3E4804F0B4F86C
:10889000044686F31188BFF36F8F58B13A4BD3E883
:1088A000EF2F013AC3E8E12F0029F8D18DB120461E
:1088B00004F0BEF925B9354B1B680BB1FFF718FF63
:1088C000304804F097F8051C18BF01252846BDE87C
:1088D000F88F2F4B1B78ABB9237ADB0712D404F047
:1088E000B6F98146204604F083F90146484604F073
:1088F00096F80746274B284ADFF8B4B09B1AC3F313
:10890000C90A37B9254E264F4FF00008BF1B3F114B
:1089100033E0B7FA87F6C6F11F063146204604F069
:108920006AF9204B0246984202D31F4B984213D358
:108930001046FFF78BFF78B91C4B9A420CD00123ED
:1089400063F3020860F3C5086AF38F1843464A468A
:108950003146584604F0A4F8012303FA06F627EA44
:108960000607CEE773685B7923B1336821461B683D
:108970003046984708F101081036B845F2DB96E713
:108980004803012014000120080001200C000120F0
:1089900049030120ECDC0000DCDC00001CDD0000F1
:1089A0002CDD000018DA00001CE60000AFDE00003D
:1089B000CDDE0000F8B50E4F3D7875B9FFF7EEFE3D
:1089C0000C4C0D4E361B3611B54207DB0020FFF76D
:1089D0004DFF0028FAD101233B70F8BD63685B7935
:1089E0001BB1236820461B69984701351034EBE71B
:1089F000490301201CDD00002CDD000008B5FFF755
:108A0000CDFE03F041FB0B4B186030B10A4B1B68E5
:108A1000092B02DD094803F03DFB084C0020FFF75D
:108A200025FF0028FAD14FF0FF31204603F058FB14
:108A3000F4E700BFD00001200800012078480120A1
:108A4000244B70B51B68418105469847224CE8606D
:108A5000D4E8EF3F0133C4E8E23F002AF8D14FF0F9
:108A60002003EFF3118683F31188BFF36F8F1B4848
:108A7000294603F0B5FF86F31188BFF36F8F184BBB
:108A80001A787AB14FF02003EFF3118483F3118841
:108A9000BFF36F8F0020FFF7E9FE84F31188BFF367
:108AA0006F8F70BD0F49236809680029F9D0012B29
:108AB00006D1BDE870404FF47A710B4803F034BD25
:108AC0000A2BEED1084804F07AFFBDE87040074851
:108AD00003F0E0BABC470120080001201400012087
:108AE00049030120D00001201C000120784801200A
:108AF00007B504380190D0E8EF3F5A1EC0E8E12FD7
:108B00000029F8D1012B03D101A9034802F090FEFE
:108B100003B05DF804FB00BF480001208023202241
:108B20000149024804F00DBEB8370120D4000120ED
:108B3000002373B50A4E02AC44F8043D0120FFF750
:108B400095FE0546FFF7F6FD00222146304602F06D
:108B500041FE08B1002DF1D1019802B070BD00BFF7
:108B6000D400012007B5002202A941F8042D0548D0
:108B700002F030FE10B1FFF7DBFF0190019803B067
:108B80005DF804FBD4000120F0B5047A457A85B085
:108B900014F0010401904FEA151510D0019B1A7AC8
:108BA000920706D55B6904AC184D44F8043D039B5D
:108BB0002BBB01A9154802F03BFE05B0F0BD002D0E
:108BC000ECD0264617E0314604F015F80746FFF7CB
:108BD0003DFE78B13CB9019B2946186903F01FFF9F
:108BE00004460028DAD024FA06F3DB0702D538461B
:108BF000FFF77EFF0136AE420198E4D3CEE71E6850
:108C00002146284602F014FE0396D0E7D400012046
:108C10000EB403B503AB53F8042B0146044801938B
:108C200003F033FD002002B05DF804EB03B07047A1
:108C3000F5CF00002DE9F04F11F0020485B0064693
:108C400090469DF8387001F0010901F0080507D041
:108C500011F0440F37D11A463249FFF7D9FF0446C5
:108C6000B9F1000F0AD0304B304953F82720304B70
:108C70003046002A08BF1A46FFF7CAFF3DB12D4B08
:108C80002D4953F827203046FFF7C2FF0546B8F1BB
:108C9000000F44D0012303FA07F7284B17F0100FF9
:108CA000274F18BF1F46BDF840109DF83C00FFF746
:108CB0004DFD394602463046FFF7AAFF28442044BE
:108CC00005B0BDE8F08F1F4A116831B31E4A4FF45A
:108CD000616E14684FF47A7CB3FBF4F3B3FBF1F4E8
:108CE000B4FBFEF20EFB124E01FB14340CFB04F439
:108CF000B4FBF1FB4FF03C0A01FB1B440CFB04F4FA
:108D0000BEFBFAF3B4FBF1F1CDE901B10AFB13E1CB
:108D100000910E49FFF77CFFA1E708469FE7084F47
:108D2000C1E700BF3FDF000058DD000064DF000046
:108D300031DF00006CDD000067DF000036DF00007F
:108D40003ADF0000F0000120F400012048DF0000BD
:108D500038B50C46E107054603D5084A0849FFF730
:108D600057FFE20608D4A3062846BDE838404CBFAA
:108D700004490549FFF74CBF38BD00BF31DF000093
:108D800064DF0000A3DF0000A2DF00002DE9F04750
:108D90009846089B0446DD060E46174605D49906FC
:108DA0004CBF29492949FFF733FF0025DFF8A4907C
:108DB00045452ADB0025DFF8A080DFF8A090DFF82A
:108DC00094A0AF422ED9725D49462046FFF720FF9E
:108DD0000135102D1FD11E492046FFF719FF002530
:108DE000DFF87080DFF87890AF4227D9725D49468E
:108DF000A2F120035F2B28BF2E222046FFF708FF99
:108E00000135102D13D1BDE8F08749462046FFF704
:108E1000FFFE0135CCE76A07D3D151462046FFF764
:108E2000F7FECEE741462046FFF7F2FED0E76B079C
:108E3000DAD141462046FFF7EBFED5E74146204612
:108E4000FFF7E6FEDCE700BFA3DF0000A2DF0000C3
:108E50000DDF00000BDF000009DF000003DF000072
:108E60000FDF00002DE9F04717460A7A8B7AD243CC
:108E700013F007048AB005460E46D2B21BD04989CA
:108E8000C3F3C20389090291CDE9004302F0010254
:108E9000F3683946FFF7CEFE8146337ADA070CD401
:108EA0002946304603F03CFF4CB32246394628465B
:108EB000FFF74EFF23E0A146EFE734BB2746EB6800
:108EC00006AA0693A9683B46304603F015FF069AAA
:108ED0006B681A603AB1AB68134413F8014CA4F103
:108EE0000A035C425C41284604F077F8069B1F4465
:108EF000002BE4D11CB115492846FFF789FE28460E
:108F000004F06BF80AB0BDE8F087304603F09FFE2E
:108F10000F4902462846FFF77BFE4FF000084FF04E
:108F2000100A05AA434606A93046CDF814A003F05E
:108F3000E3FE059A002AB8D04B46009706A92846BA
:108F4000FFF724FF059B9844EBE700BF12DF00000A
:108F500064DF000073B5D0E900435D6842F20F732F
:108F60008B4228BF0B460D4A0521684601F03CFFA5
:108F700006462B4620460422094903F0C4FE2B4630
:108F800032466946204603F0BEFE2B4617220549AD
:108F9000204603F0B8FE02B070BD00BF88E50000B7
:108FA0002CDF000014DF000001230021074A10B568
:108FB000074C1360A04204D801B11360054B186040
:108FC00010BD40085B000121F4E700BFF400012060
:108FD00040420F00F00001200122034B1A70034BA6
:108FE000034A1A60704700BF4B03012008010120AB
:108FF0004C03012008B5034803F0EFFF0122024BA8
:109000001A7008BD98DD0000630401200148FFF7D5
:10901000A1BF00BF98DD000010B50C46084603F064
:10902000DEFD214604480A22FFF71CFF2046BDE86A
:10903000104003F0FDBD00BF98DD0000044B1B781D
:109040001BB142F2107004F054BC0A2002F0F4BFCD
:10905000630401202DE9F74F5B4E814633780F46BC
:1090600043B98246594C09EB07039A4540D3AAEB12
:1090700009001DE00A24DFF86C81554D337823B9CF
:109080004FF0FF31404602F001FC3A4649460020CD
:1090900000F0B6FA3378824613B9404602F068FC15
:1090A000BAF1000F18D001232B7033783BB9384642
:1090B00003B0BDE8F08F5CB92C704FF0FF34002096
:1090C00000F01CFB0028F2D02B78002BF3D1EEE748
:1090D000013CFFF7B3FFF2E72B7813B1013C04D159
:1090E0002C702B78002BC9D1E1E7FFF7A7FFF8E739
:1090F0001AF8012B23680A2A5FD1364D0A265A1B1B
:10910000012A4FF00D0204BF01332360236803F8E6
:10911000012C1E705A1C304B2260D3F800B0BBF1FA
:10912000000F25DD2D4B196811BB2A49BBF1630FD8
:10913000A2EB050201F117000193D846A8BF4FF03A
:10914000630804F0CAF817222549224804F0DCF825
:109150002268019B173222600122BBF1090F1A60BD
:109160001DDC202308F130086B7585F81480EB7442
:109170004FF0FF311B4802F089FB22681549521B52
:10918000002000F03DFA0546164802F0F1FB124BB4
:109190007DB91A6801321A600E4B236063E798FBB1
:1091A000F6F306FB1386303330362B756E753E238F
:1091B000DDE700221A60094BEDE70B498B423EBF09
:1091C000591C21601A704EE7630401200801012038
:1091D0004B0301204C030120000101200401012068
:1091E0008DDF00009C4801204B04012010B5044C89
:1091F0002046FFF701FA204601F0F0FD002010BDE7
:10920000059200002DE9F34106460324154F164D43
:109210008DF807004FF0FF31384602F037FB01228E
:109220000DF10701002000F035FA8046384602F0C3
:109230009FFBB8F1000F05D001232B70304602B020
:10924000BDE8F0812B78002BF8D0013C07D004F06A
:109250004AFB0028DED1022002F0EEFEDAE72C7095
:10926000ECE700BF9C4801206404012003682DE95D
:10927000F041D0F808C005469F68CEB24AB10C2331
:1092800073435CF803309A425BD013B11B68002B28
:10929000F9D14FF02003EFF3118083F31188BFF36E
:1092A0006F8F0C2171430CEB01031C7A0134E4B283
:1092B0001C7280F31188BFF36F8F22B34FF0030E3F
:1092C0002248C0F808E3587AA0B94FF0200EEFF317
:1092D00011888EF31188BFF36F8F1060D3F804E00C
:1092E000BEF1000F20D15A604CF8012088F311889C
:1092F000BFF36F8F0321154BC3F8041318B1D2E9E4
:10930000013128469847012C0CD14FEA061857F82E
:1093100008306BB901224744BB7A03F1804303F55F
:10932000A0431A6000200EE0CEF800205A60DDE76E
:10933000284698470028EDD13146284603F0C1FE63
:10934000F0E76FF00F00BDE8F08100BF0050004073
:1093500010B5002204460121052000F085FA052001
:1093600000F072FA0222074B0020C3F818250322EE
:10937000C3F80423A368C3E90000A368C3E903009A
:1093800010BD00BF0050004008B5104B1A6862B114
:109390000F4AD2F80423D10707D500220D481A60DE
:1093A0008368597A09B903F08CFE0B4B1A6862B1D5
:1093B000074AD2F80423920707D5002201211A6038
:1093C0000448BDE8084003F07CBE08BD00510040E1
:1093D00000500040244801200451004000220D4B61
:1093E000C3F840214FF02002EFF3118182F311887E
:1093F000BFF36F8F084AD3F804051368C01A20F032
:109400007F400344136081F31188BFF36F8F02F034
:10941000F3BF00BF005001403001012070B5154876
:1094200002F03EF810B3436801211B6898470024FE
:1094300001264FF480334FF400120F4D3146C5F82A
:109440000845C5F84065C5F804330C4B15201C6071
:109450000B4BC3F88021224600F006FA152000F0DD
:10946000F3F92046074B1E602E6070BD4FF0FF30B1
:10947000FBE700BFBBDF000000500140405101404E
:1094800000E100E00850014070B5264EB0F1FF3F0A
:1094900008BF30464FF02003EFF3118483F31188A7
:1094A000BFF36F8F204BD3F80455204B1B68EA1A8B
:1094B00022F07F42B2F5000F1AD2411E21EAE1717B
:1094C000B142A8BF3146501C0844B04294BF18189E
:1094D0009819451B25F07F45134A20F07F43022D44
:1094E000C2F8403506D984F31188BFF36F8F70BD81
:1094F0000021E8E7D2F804350D49C31A23F07F4371
:109500005D1E8D4205D94FF400120A4BC3F80021AD
:10951000E9E7012B02BF023020F07F40C2F840058E
:10952000E1E700BFFEFFFF000050014030010120D5
:10953000FEFF7F0000E100E04FF02002EFF3118317
:1095400082F31188BFF36F8F064AD2F80405064AEA
:109550001268801A20F07F4083F31188BFF36F8F69
:10956000704700BF00500140300101204FF0200340
:10957000EFF3118283F31188BFF36F8F0649074B16
:109580000868D3F8043582F31188BFF36F8F1B1A74
:1095900023F07F4318447047300101200050014000
:1095A000032310B5104C114AC4E90433104BA261D7
:1095B000E3614FF4805322660E4A23626266002301
:1095C00010220D49E01DA3626362E3622367E36634
:1095D0006367A26603F039FE0849204603F035FEB2
:1095E0002023A37110BD00BF34010120E5DF00007E
:1095F0007504012065040120EEDF0000F2DF0000A9
:109600002DE9F04707461820214D144600FB07526C
:10961000936A566A8846B34233D8126AA2EB0609A7
:1096200009F1FF32944211D84FF0180907FB099352
:109630002B44586822464146304403F065FE09FB3E
:109640000755344401206C62BDE8F08713449C4206
:109650001BD807FB000005EB000ADAF804004A46B5
:10966000304403F051FEB4EB090406D0224608EB67
:109670000901DAF8040003F047FE182303FB07553D
:10968000E0E7013B9B1BA342CED20020DCE700BFFA
:1096900034010120F8B51823174C00FB033503FBF8
:1096A00000402544C46A0F46012C164611D003D34E
:1096B000022C1BD000240AE0284603F02AFD864233
:1096C00005D832463946284603F031FD3446204657
:1096D000F8BD284603F01DFD8642344628BF0446E7
:1096E00039462246284603F022FDF0E72846BDE829
:1096F000F84003F039BD00BF340101201823034AAC
:1097000003FB00239A6A586A801A704734010120CB
:1097100004488168406A884203D003494FF0805270
:109720000A6070470803012004ED00E012498A68CE
:109730004FF028001044EFF3098C80E8F01F202040
:1097400080F31188BFF36F8F0C4F4FF000664A6AA9
:109750008A603E60506E0023536680F3118804B522
:10976000104603F03EFDBDE8044002F1280090E8F9
:10977000F01F8CF3098870470803012004ED00E016
:109780001EF0040F0CBFEFF30880EFF3098081692E
:1097900011F8021C0229FFD001B503F017FD01BD2D
:1097A000014910220A60704710ED00E0404080F34C
:1097B000118830BF704700BFEFF30880EFF30981D5
:1097C000724601B500F004FB01BD00BF30BFFFF7DA
:1097D000FDBF00BF01B572B60B4A106A00281EBF5C
:1097E0000021116203F0ABFF62B6EFF30580A0F138
:1097F00010004FEAC0000549014409C99847BDE877
:1098000001400349084700000803012018DA00005E
:1098100011970000094A0A499368096858669966D1
:1098200008494B6843F080534B60002383F3118851
:10983000BFF36F8F9368986E704700BF08030120D5
:1098400060DE000000ED00E043B2002B08DB0122E7
:1098500000F01F0002FA00F0024A5B0942F8230000
:10986000704700BF00E100E043B2002B01F10101AD
:10987000A8BF03F160434FEA4111B8BF054BC9B21D
:10988000ABBF03F5614300F00F0083F800131954D8
:10989000704700BF14ED00E073B51E460A9B0546F5
:1098A0000093099B8C1804F02BF80B4AA4F12003B9
:1098B00023F0070322F001029A61069A1E605A60A3
:1098C000079A9A60089ADA604FF08072DA61AB64A6
:1098D00000236B6602B070BD91C90000F8B5054663
:1098E0000C4617461E4600F0BFFB0A4B3C44284678
:1098F0009D6024F0070403F074FC304684F309886B
:10990000002163B681F31188BFF36F8F002200231B
:1099100003F03EF808030120F7B507460C4600297E
:109920003DD001264FF00003204A214D66F302038B
:10993000AD1AC5F3C9056FF3C50365F38F13ADF811
:109940000030D1E901231B48096803F0C1F84FF04A
:10995000000366F302036FF3C50365F38F13ADF8DD
:109960000030D4E90423E168134803F0B1F84FF064
:10997000000266F302026FF3C50265F38F12E1691C
:109980000E4803F079F84FF0000266F302026FF31D
:10999000C50265F38F12A169094803F06DF82146ED
:1099A000384603B0BDE8F04001F0A0BDDCDC0000AB
:1099B000FCDC0000F9DF000028E0000057E00000B8
:1099C00066E0000008B5084B084A23F07F03936067
:1099D000BFF34F8FBFF36F8F01F00EFE01F016FE45
:1099E00000F010FB01F050FE0080000000ED00E0F0
:1099F00002F0F0FF202080F3118808484FF4006146
:109A0000401880F30988EFF314800221084380F3A3
:109A10001488BFF36F8FFFF7D5FF0000B81D01203A
:109A200070B54FF000010126404B414C66F3020136
:109A3000E41A6FF3C501C4F3C9043E4D64F38F11FA
:109A40003D4803F00CF8AA6A92010AD54FF00001D4
:109A500066F302016FF3C50164F38F11374802F01A
:109A6000FEFFAB6ADB010BD54FF00001012363F36E
:109A700002016FF3C50164F38F11314802F0EFFF6B
:109A80002C4DAA6AD6020BD54FF00001012363F3D7
:109A900002016FF3C50164F38F112A4802F0DFFF62
:109AA000AB6A18030BD54FF00001012363F30201E9
:109AB0006FF3C50164F38F11234802F0D0FF1D4DF1
:109AC000AA6A51030BD54FF00001012363F3020191
:109AD0006FF3C50164F38F111C4802F0C0FFAB6A3D
:109AE0009A030BD54FF00001012363F302016FF3DA
:109AF000C50164F38F11164802F0B1FF0D4DAB6A3A
:109B0000DB030BD54FF00001012363F302016FF378
:109B1000C50164F38F110F4802F0A1FFAB6A00206A
:109B20006FEA03436FEA1343AB6270BDDCDC0000F5
:109B3000FCDC000000ED00E0F4E100000CE20000BD
:109B40001FE2000039E2000063E2000081E2000051
:109B5000A6E20000C0E200002DE9F0410E464FF001
:109B600001084FF000013D4B3D4C68F30201E41A3F
:109B70006FF3C501C4F3C9043A4D64F38F1107466E
:109B8000394802F06CFFAA6AD1060AD54FF00001ED
:109B900068F302016FF3C50164F38F11334802F0DB
:109BA0005EFFAB6A1A070BD54FF00001012363F388
:109BB00002016FF3C50164F38F112D4802F04FFFCE
:109BC000284DAB6A9B0720D54FF001084FF00001EC
:109BD00068F302016FF3C50164F38F11254802F0A9
:109BE0003EFF696BAB6A18060FD54FF0000268F3B1
:109BF00002026FF3C50264F38F121F4802F03CFFAC
:109C00001FB1AB6A23F08003AB62164DAA6AD2077C
:109C10000BD54FF00001012363F302016FF3C5017F
:109C200064F38F11154802F01AFFAB6A9B060BD53F
:109C30004FF00001012363F302016FF3C50164F3E8
:109C40008F110F4802F00BFF0020064B9A6A9A6AA8
:109C500042F0FF029A623070BDE8F081DCDC000067
:109C6000FCDC000000ED00E01CE1000032E100003F
:109C700065E1000078E1000090E10000A6E100004D
:109C8000C5E100002DE9F0410E464FF001084FF00C
:109C90000001444B444C68F30201E41A6FF3C50120
:109CA000C4F3C904414D64F38F110746404802F0E4
:109CB000D6FEAA6AD1040AD54FF0000168F302016A
:109CC0006FF3C50164F38F113A4802F0C8FEAB6A26
:109CD0001A050BD54FF00001012363F302016FF366
:109CE000C50164F38F11344802F0B9FE2F4DAB6A01
:109CF0009B0520D54FF001084FF0000168F30201E9
:109D00006FF3C50164F38F112C4802F0A8FEA96B14
:109D1000AB6A18040FD54FF0000268F302026FF32C
:109D2000C50264F38F12264802F0A6FE1FB1AB6A8B
:109D300023F40043AB621D4DAB6A59050BD54FF0C0
:109D40000001012363F302016FF3C50164F38F1176
:109D50001C4802F084FEAB6A13F4807314D04FF0F9
:109D60000001012363F302016FF3C501164864F398
:109D70008F1102F074FE00200C4A936A43F47F4373
:109D800093623070BDE8F081AA6A9204F3D54FF077
:109D90000001012262F3020163F3C50164F38F1134
:109DA0000A48E6E7DCDC0000FCDC000000ED00E037
:109DB00094E00000AAE0000065E10000BBE00000C4
:109DC000D4E00000E9E0000004E10000C5E100008B
:109DD0002DE9F041704B8AB05F680646884614460C
:109DE000C7F30807002585F31188BFF36F8F02F0D2
:109DF0007F43B3F17F4F2CD112F0010329D16206CA
:109E000004D4230723D54646002512E001224FF053
:109E1000000162F3020163F3C501604A604B6148CF
:109E20009B1ADB0863F38F1102F019FE14F004058E
:109E3000E9D100238DF80730FB1E092B00F28E803C
:109E4000DFE803F00972766F8C8C8C8C8C7A01259C
:109E5000EFE72E46EDE74FF001084FF00001002438
:109E60004E4B4F4F68F30201FF1A6FF3C501C7F362
:109E7000C90767F38F114C4802F0F1FD464A8DF88F
:109E80000740D36A13F0020324D04FF0000168F3B7
:109E9000020164F3C50167F38F11444802F0DFFD4E
:109EA0009DF807309BB92022314602A803F02CFA16
:109EB000099B002D6AD0C3F3080222B96FEA53232D
:109EC0006FEA4323099302A92046FFF725FD0AB054
:109ED000BDE8F081D46A14F08044E4D04FF0000172
:109EE00068F3020163F3C50167F38F11304802F094
:109EF000B6FD304B1B7833B140460DF10701FFF73B
:109F00002BFE0446CCE72C4B1B782BB140460DF1C1
:109F10000701FFF7B7FEF4E7284B1C88A4B2002C1A
:109F2000BED0FFF77DFDECE70DF107010020E6E76D
:109F30000DF107010020ECE701234FF00001174A63
:109F400063F30201164B6FF3C5019B1ADB0863F341
:109F50008F111B4802F083FD0024A1E701224FF07E
:109F600000030E4962F302030D4A1648521A1649BD
:109F7000D2086FF3C50362F38F130F2FC8BF0146DA
:109F8000A7F11002114802F08BFDE5E723F4FF73FF
:109F900023F0010396E700BF00ED00E0DCDC0000E9
:109FA000FCDC0000EBE200000EE3000025E3000013
:109FB00046E3000028ED00E029ED00E02AED00E096
:109FC00065E30000B0E300009BE30000C9E300008C
:109FD000024A536943F010035361704700ED00E0FB
:109FE000BFF34F8F0549064BCA6802F4E062134382
:109FF000CB60BFF34F8F00BFFDE700BF00ED00E077
:10A000000400FA05002320210348C2180133452B20
:10A0100082F80013F9D1704700E100E038B5054639
:10A020004FF02003EFF3118483F31188BFF36F8F98
:10A0300001F076FE0A4B9B68AB420BD1094B5A6884
:10A04000C2F3080212B92046FFF7E4FB5A6842F057
:10A0500080525A602046BDE8384003F0CABB00BFBA
:10A060000803012000ED00E010B50E4B88B002930C
:10A070000D4B0E4C03930E4B08A8049302AB40F813
:10A080001C3D0C4A2346012100F056F9002307939A
:10A09000094B0121E41A05A80593069400F056F92E
:10A0A00008B010BD000001200000000000000720E3
:10A0B00006000100000001200000012010B50B681F
:10A0C0000C7A23F01F0304F01F021A43CB686409C3
:10A0D00023F01F03044943F0010343EA440388606B
:10A0E000CA600B6110BD00BF90ED00E008B54FF0F5
:10A0F00000020123084963F30202084B6FF3C50213
:10A100005B1ADB08014663F38F12054802F0B4FCCA
:10A110006FF0150008BD00BFDCDC0000F4DC0000BF
:10A1200026E400002DE9F04F074688461446002635
:10A13000604D85B0464541DA57F82630D3F8049093
:10A14000B9F1000F5DD0B9F11F0F24D919F01F0F1D
:10A1500021D1D3F800A01AF01F0F1CD1504603F0F4
:10A160006BF8834609EB0A00013803F065F8834574
:10A1700028D06FF0150B01234FF000024E4963F316
:10A1800002024E4B6FF3C5025B1ADB0863F38F12BA
:10A1900059464B480EE001234FF00002464963F355
:10A1A0000202464B6FF3C5025B1A3146DB08454895
:10A1B00063F38F1202F060FC6FF01504204605B0C7
:10A1C000BDE8F08F1BF1160FD5D0631E5B45D2DBC7
:10A1D000C5F808B0E868C5F808B02B6957F826102C
:10A1E00020F01F0043F01F0AD1E900321A449842C0
:10A1F00002F1FF3918D1CA4505D15FFA8BF002F0A0
:10A20000F8FF013696E7C5F808B0EB6822F01F02A8
:10A2100003F01F031A43EA60E0B202F0EAFF10F114
:10A22000160FC9D0441CECE7C5F808B02A69013BF9
:10A2300023F01F0302F01F021343CA45E0B22B6153
:10A24000EBD002F0D6FF10F1160FB5D0C5F808B06C
:10A25000EA689DF808300AF1FF3A62F304038DF8CA
:10A2600008302B699DF808205B0863F3471257F804
:10A2700026308DF80820D3E900130B44009323F017
:10A280001F03441C5344A3EB0903E4B223F01F0350
:10A290000F2C039308D92046FFF728FF10F1160F63
:10A2A000044689D00134ACE769462046FFF706FF33
:10A2B000F8E700BF90ED00E0DCDC0000F4DC00001B
:10A2C00003E40000E0E300000522034B5A60BFF303
:10A2D0004F8FBFF36F8F704790ED00E0BFF35F8F3C
:10A2E0000022014B5A60704790ED00E070B50E4DB2
:10A2F0002E68102E15D80024FFF7F0FF0B4B0C4AE8
:10A300001A63A64205D10B4B1E70FFF7DDFF00203C
:10A3100070BD6968204601EB0411FFF7CFFE0134E0
:10A32000EFE74FF0FF30F3E7DCDD000090ED00E0F9
:10A33000AAFF44007514012010B5034C2278FFF7E2
:10A34000F1FE207010BD00BF751401202DE9F74FFC
:10A35000894607460026DFF89080DFF890A0214C60
:10A360004E4519DAD7F804B0BBF1000F36D03B6880
:10A370001846019302F060FF019B05460BEB0300BA
:10A38000013802F059FF1423854203FB06F306D07F
:10A390006FF0150248F8032003B0BDE8F08F15F107
:10A3A000160F48F80350F7D09AF80020AA42F3DDC0
:10A3B000A5604344A560E068197B60F3040119734C
:10A3C0002169187B490861F347101873E26822F08D
:10A3D0001F025A60226922F01F021A6101360C37EF
:10A3E000BEE700BF90ED00E0DC0101207514012004
:10A3F00070B50C4B0E461C780546234600210A4AD0
:10A400000F2B0BDD094B191D1868FFF757FE22466D
:10A4100031462846BDE87040FFF784BE9360116165
:10A420000133EDE77514012090ED00E0DC0101201F
:10A430002DE9F04F1E4600239DB0CDE902010193A6
:10A440001078531C069358B1252800F08980039991
:10A45000029B9847013040F00B844FF0FF3301938B
:10A4600001981DB0BDE8F08F232C70D065D8002C6A
:10A47000F6D0202C0C9B08BF01230C93CDF818803C
:10A48000DDF81880BB4818F8014B214602F0FAFEAF
:10A490000028E9D12A2C6AD13268331D002A07929C
:10A4A000BEBF5242079201221E46B8BF0D92069AC5
:10A4B000547802F102082E2C7ED198F800302A2B15
:10A4C00077D1356808F10108043698F8004008F1A2
:10A4D00001082146A848274602F0D4FE00286ED085
:10A4E00008F10103682F069398F8004007D1682C03
:10A4F00005D1482708F1020398F801400693672C1C
:10A500007CD8652C80F03A81472C5CD8452C80F0B3
:10A510003581002CA4D0252C00F0A683039925209A
:10A52000029B9847013098D003992046029B984798
:10A53000013092D0019B02339CE32D2C0DD0302CA6
:10A5400008D02B2C099B08BF0123099396E7012310
:10A55000059393E70123089390E701230D938DE77B
:10A56000002308930C9309930D93059388E7A4F1B6
:10A570003003092B07909ED80A22DDF8188018F8BE
:10A58000014BA4F13003092B95D8079B02FB034430
:10A59000A4F13003CDE90683EFE7904601FB0535D2
:10A5A000303D424612F8013BA3F130000928F4D9AE
:10A5B0008BE700250A21F4E74FF0FF3589E7CDF856
:10A5C000188007469BE7632C59D021D8582CA5D179
:10A5D000331D6F2C0493316815AF40F01B83059B2E
:10A5E000002B00F00B8330238DF85430002940F00D
:10A5F0000E838DF855108B46012726E0702C00F055
:10A60000E88227D86E2C00F0CF82E1D8692C85D162
:10A610003468331D002C049380F29E802D23614208
:10A620008DF854300DF1550738460A2202F0BAFE73
:10A63000099B074415A83F1A002B40F01E830C9B72
:10A64000002B40F01A834FEAD47B002DC0F21A830E
:10A6500015AE1EE0752CBBD0782CB9D0732C7FF4CE
:10A660005DAF002DB8BF6FF000450027331D366881
:10A670000493BD4240F0BD820025AB4609E04FF097
:10A68000000B01275D46331D049333681CAE06F8AA
:10A690001C3DA5EB070A0025A846A946DA442AEA8C
:10A6A000EA7A079B0AEB07041C1B0D9B13B9002CCD
:10A6B00000F3078306EB0B039E4240F004835346EE
:10A6C00013F1FF3380F00B83A7EB0B07B9F1000FF9
:10A6D00000F02A833078F219A0F130010929A2EBA9
:10A6E000060340F207834A46002A40F00E83A3EB9C
:10A6F0000909B8F1000F18D006EB090316F8012B71
:10A70000079303991046029B0592984701303FF446
:10A71000A4AE059A079B2E2AA3EB0609EED1434669
:10A72000002B00F30383A9EB08099DB1307806EBF9
:10A730000908A0F13003092BA8EB060940F20383B6
:10A740002E2800F00083A846B8F1000F00F3048320
:10A75000A9EB0509B14412E3099B23B12B238DF822
:10A76000543021465EE70C9B0BB12023F7E72146CE
:10A7700015AF59E74CE4000052E40000073626F01C
:10A780000706D6E90001C202904606F108030493C9
:10A79000CB0243EA5053002823F0004971F1000333
:10A7A000C1F30A56CDE9108942DA2D218DF85410F3
:10A7B0000DF1550740F2FF718E4254D158EA09035A
:10A7C000A4F1410407F1030042D1192C3AD84923DE
:10A7D0003B704E237B7046230025A846A946BB70DC
:10A7E000FD7015AFC01B099B002B40F0DA810C9B5C
:10A7F000002B40F0D6819DF854B0ABF12D03D3F17E
:10A80000000B4BEB030B1CAB5B4413F81C3C08EB3D
:10A810000907303B2F44092B074400F23782089B7D
:10A82000002B00F03982079B15AEA3EB070A36E731
:10A83000099B0BB12B21B9E70C9B0BB12021B5E78C
:10A8400015AFB7E769233B706E237B706623C3E7C0
:10A85000192C99BF4E2341226E23612294BF3B7075
:10A860003B707A70B8E7462C48EA060049EAE67180
:10A8700008BF662450EA010300F0DA80002E7AD087
:10A88000DDE910231046A6F2FE38002643F0004111
:10A890000DF1700969E90C0118F1020F7ADB6FF014
:10A8A000004A4FF0000BB8F1000F00F3A48010A88D
:10A8B00008F1010802F096FDB8F1040FF7D1002D60
:10A8C00004F0DF03B8BF0625472B40F0B980F21C27
:10A8D00002DBB54280F2AF80023CE4B2002D00F012
:10A8E0007382059B013D002B40F06E82002DD4BF8A
:10A8F0004FF0000A4FF0010A662C40F0678215EB1A
:10A90000060840F1A380102366244FF000080F933F
:10A9100000224FF000630DF1700969E90A2318F174
:10A92000FF3880F09580DDE91023DDE9120112EB9C
:10A93000000843EB0109CDE9108909F070484FF098
:10A94000000958EA090306D010A802F05EFD10A81D
:10A9500002F048FD0136662C40F0C480002E7DDCFC
:10A9600030233B70059B07F1010B002B40F08D80DD
:10A97000994685E0013E18EB080849EB0909B8F152
:10A98000000F79F10003F5DACDE9108978E7484640
:10A9900002F028FDDDE910A000230B9300230A90AC
:10A9A000BC4ADDE90ABC634508BF5A4508F1010805
:10A9B000EDD305224FF0000CAAFB02AB02FB00BB5B
:10A9C000CDE910AB013E002300216FF00040994219
:10A9D00008BF584506D2BCF1000F3FF45DAFCDE98A
:10A9E00010AB59E71AEB0A0A4BEB0B0B08F1FF38D7
:10A9F0004FF0010CE7E710A802F007FDDDE91001B8
:10AA00004FF0000C08F1FF38013600239B4508BFCA
:10AA10008A4506D2BCF1000F3FF445AFCDE91001E5
:10AA200041E70018494108F1FF384FF0010CECE70D
:10AA30000026B0463BE7059BAD1B23B9662455E7CE
:10AA40004FF0000A58E74FF0000A58E76624BFE1CC
:10AA5000484602F0DAFC02F0C5FC60E7BB460F9BFB
:10AA6000002B07DD0FA910A802F0FFFC013E0BF838
:10AA7000010BF4D1059B002B40F09D81B1461E4691
:10AA8000002D04DC4FF0000820E04FF000092E22DA
:10AA90000BF101038BF80020002E00F09381002DB4
:10AAA0001EDDC6F10008A845A8BFA846A5EB08050D
:10AAB0009B4606E00FA910A802F0D7FC013D0BF859
:10AAC000010B002D02DD0F9B002BF3DCBAF1000F10
:10AAD0001ED1002315AF8BF80030ABEB070082E6E8
:10AAE0009B46CFE70FA910A802F0BFFC059B3028BA
:10AAF000387018BF06F1FF36002B3CD1002D3ADC30
:10AB000007F1010BBAF1000F48D04FF00009C84619
:10AB10001BF8012C0BF1FF33302A3DD02E2A08BF41
:10AB20009B46002504F0DF03452BD2D1002EB4BF95
:10AB30002D232B235A46B8BF7642632E02F8024BD0
:10AB40008BF801300ADD642196FBF1F301FB1366FB
:10AB500003F130000BF103028BF802000A2196FB8F
:10AB6000F1F3934601FB136603F1300030360BF826
:10AB7000020B5670ADE72E2307F1020B7B70002D00
:10AB8000C0DD0F9B002BBDDD0FA910A802F06DFCEE
:10AB9000013D0BF8010BF2E79B46B9E7D146D046E1
:10ABA000C0E74FF0010B2EE6324652F8043B682F07
:10ABB000049206D06C2F09D0482F07D1019A1A7041
:10ABC00001E0019A1A80049E069A39E4019A1A60FB
:10ABD000F9E7331D049347F63003316810220DF175
:10ABE0005600ADF8543002F0DDFB4FF0020B871C2D
:10ABF0002BE5F35D002B43D001373AE538460822B8
:10AC0000C71B02F0CFFB07444FF0000B1DE50DF111
:10AC10005500F4E7752C05D138460A2202F0C2FB34
:10AC20000746F1E7059BEBB147F630030DF15606F9
:10AC3000ADF854301022304602F0B4FB582C0BD142
:10AC40003B461A78A2F1610119299CBF203A1A707B
:10AC500013F8012B002AF4D1059BF71B07444FEA98
:10AC6000430BF2E43E46E5E703992046FFF7F0BBCD
:10AC7000019B013301930496A5E74FF0010BE4E437
:10AC80001D46FAE40025A846A946C8E515AE4FF0D2
:10AC9000000A06E53233333315AEDDF820A000E5B7
:10ACA00005930399029B202098470130059B3FF4B0
:10ACB000D4AB13F1FF33F3D2019A224401921C4624
:10ACC000F8E42346F5E705930399029B16F8010B78
:10ACD00098470130059B7FF4EFACFFF7BEBB0593AF
:10ACE0000399029B302098470130059B7FF4E8AC24
:10ACF000FFF7B3BBDDE902310592984701303FF41D
:10AD0000ACAB16F8010F059AE6E405930399029B94
:10AD1000302007929847079A013002F1FF32059BD5
:10AD20007FF4E2ACFFF799BBB946E2E405930399DF
:10AD3000029B30209847059B013003F1FF337FF4DD
:10AD4000EFACFFF78ABBDDE90231984701303FF4F1
:10AD500084AB16F8010FECE403993020029B98476E
:10AD6000013008F1FF387FF4EFACFFF776BB0399B1
:10AD700016F8010B029B984701303FF46EABA9EB2C
:10AD80000603002BF3DC019B002C5B449B46D34461
:10AD900007EB0B0301937FF716AF2344019314F1E4
:10ADA000FF34FFF410AF03992020029B9847013035
:10ADB000F5D1FFF752BB2E22B14600260BF101035D
:10ADC0008BF80020B04673E64FF0000A05F1010849
:10ADD000102398450F93A8BF984699E5014B18603A
:10ADE000704700BFC04701200CB41FB509B90DF171
:10ADF0000300CDE9020107AB069A02A905480193B9
:10AE0000FFF716FB0022029B1A7005B05DF804EBF9
:10AE100002B07047A7D4000008B5094B1A786AB988
:10AE200001212F2019700521FEF71EFD2F20FEF7AE
:10AE30000BFD4FF00042034BC3F80423002008BD74
:10AE40007614012000F002401F288ABF074B084BF0
:10AE500000F01F0003EB8000D0F8003223F44033F1
:10AE600043EA0141C0F80012704700BF0028844047
:10AE700000258440F8B5036801F01F049B680D4667
:10AE80001B79484944EA43140023D1F80423866817
:10AE9000D2B203F5A27051F82000C0F3052084421D
:10AEA00065D122FA03F0C00761D59A0002F1804211
:10AEB00002F53C32D2F8100520F00100C2F810056E
:10AEC000012202FA03F3C1F8083320460021FFF7FC
:10AED000BBFFB068E84010F0010047D0F068E840E0
:10AEE00010F0010042D07069E84010F001024AD031
:10AEF000B369EB40DB073ED43369F269EB4022FAD9
:10AF000005F503F0010305F00105AB420CBF022576
:10AF100001250022234E02F5A27356F8230010F0FB
:10AF200003002AD1970007F1804303F53C33D3F89F
:10AF30001015240221F44F3121F44071C3F810158B
:10AF4000D3F8101504F47C5444EA05450D43164922
:10AF5000C3F81055C851D3F8101541F00101C3F8DA
:10AF60001015012303FA02F2C6F80423F8BD0133D9
:10AF7000082B8ED1A9E70325CBE70132082ACAD1D5
:10AF80006FF01200F2E7F169336920464B4023FA73
:10AF900005F515F0010F0CBF03210221FFF754FF47
:10AFA0001046E3E700F0024000F102402DE9F74FC0
:10AFB0008046856803F47040B0F5804F1E4648D047
:10AFC0002BDCB0F5805F3CD0B0F5405F3DD058BB86
:10AFD00006F44077B7F5807F3DD0A7F50074634253
:10AFE0006341012919BFD4B2A1464FF01F090024C3
:10AFF0004FF0010A06F0010C4FEA4C0747EA0C0734
:10B0000047EA002040EA8307DFF8CCB0314BA14586
:10B0100023D2002003B0BDE8F08FB0F5E04F16D08A
:10B0200005DCB0F5A04F0ED06FF01500F2E7B0F5DB
:10B03000404F04D0B0F5504FF6D10720C8E70620A6
:10B04000C6E70120C4E70320C2E70420C0E70520CB
:10B05000BEE70220BCE70323C3E7D8F80020019332
:10B060009268117904F01F0242EA41121F2ACABFF6
:10B070005946194602F01F02803241F82270A96831
:10B080000AFA04F2B0074CBF11439143A960696901
:10B09000B0064CBF114391436961A96970064CBF6A
:10B0A00011439143A961296970074CBF1143914332
:10B0B0002961E96930064CBF0A4321EA0202EA61CC
:10B0C00021464046FFF7D6FE0028A3D10134E4B262
:10B0D000019B9CE70025844000288440F7B50025AB
:10B0E000CDE90055244E346844B1244802F07CFA7E
:10B0F0000090234802F078FA019035600022012682
:10B100009646204DDFF880C0D5F8043306FA02F1E8
:10B11000194218D002EB0C0189000B689BB102F5B3
:10B12000A27355F8233002AFC3F3403007EB800021
:10B1300050F8087CC3F3042306FA03F33B4340F8BA
:10B14000083CC1F800E00132082ADDD1009911B1B4
:10B150000A4802F013FA019911B1094802F00EFAF7
:10B1600044B1064802F068FA054803B0BDE8F04073
:10B1700002F062BA03B0F0BD7CF1024054480120F5
:10B180006048012000F0024040BC0010F0B54B794F
:10B19000012B2DD0032B28D110248B79032B24D104
:10B1A000CE792EB1012E20D103689B681B79E3B1C3
:10B1B0000B79012B1ED020D3022B16D100220E2595
:10B1C00047F6122C03689B681F680B68634578D0AC
:10B1D00030D8B3F5965F6ED01BD8B3F5167F58D034
:10B1E0000ED8B3F5967F00F081806FF022005EE00C
:10B1F0000024D2E74FF48072E1E700221546DFE732
:10B20000B3F5966F54D0B3F5166FEED14FF41D23FE
:10B2100041E0B3F5615F50D004D8B3F5165FE4D1D7
:10B22000344B38E0B3F5964F49D0B3F5E14FDCD15C
:10B23000314B30E0B3F5E13F4CD012D84DF6C02C85
:10B24000634541D005D8B3F5164FCED14FF41D0359
:10B2500021E0B3F5614F3AD0B3F5963FC5D1274B06
:10B2600019E0B3F5E12F3BD009D8B3F5613F34D0F5
:10B27000DFF898C06345B8D14FF080630BE0B3F5B9
:10B28000612F30D0DFF888C06345AED14FF08053D6
:10B2900001E04FF41C33C7F82435324383682C4354
:10B2A000224303C9C7F86C2583E803000020F0BDE2
:10B2B0004FF49E23EFE7124BEDE7124BEBE7124BF7
:10B2C000E9E74FF40003E6E74FF46503E3E74FF4E3
:10B2D0006B03E0E74FF0EB73DDE74FF06C73DAE7F9
:10B2E0004FF0E863D7E74FF07063D4E74FF4A03333
:10B2F000D1E700BF0050270000C0750000903A0160
:10B3000000B0130000F03A0000A04E0090D00300FF
:10B3100040420F00026870B59268184B14684FF4F1
:10B320008012856803219A6014260022C3F8501207
:10B33000C3F85822C4F80C651626C4F814654FF4F7
:10B3400000269E60C3F84C12C3F854221323C4F89D
:10B35000083515232946C4F81035FFF717FF58B9EB
:10B360000823C4F800351D440123C4F81001C4F8B3
:10B370003455C4F83835236070BD00BF00258440C3
:10B3800008B5FDF717FB01234FF00001074A63F3EF
:10B390000201074B6FF3C5019B1ADB08054863F3F5
:10B3A0008F1101F05CFB0020FEF71AFEDCDC0000D0
:10B3B000E4DC00008AE400002DE9F0430025214C84
:10B3C000214E54F8048CDFF8889085B0A84503D846
:10B3D000002005B0BDE8F083636A96E807001F68A7
:10B3E00001AB83E807000C221946384601F065FFDF
:10B3F00090B98FB1636A21691B681A6991420BD1B8
:10B400009A69A169914207D8E169914204D96269B8
:10B410005B6932EA03030AD0276A67B10B4801F07F
:10B42000AAFA404080F311884FF0040002DFE3687D
:10B4300001351C44CAE7484601F09DFA636A1F6063
:10B44000F5E700BF3C82000030DD0000A7E400000B
:10B45000D0E40000044BD3F85825044B02F001025D
:10B46000D340034A13607047005000400020A107FA
:10B47000D047012070B50026084B53F8204001301A
:10B4800053F82050A54200D870BD236820465B6861
:10B49000984700B166600C34F4E700BF4CDE000052
:10B4A000104B70B505461E460F4C9C4204D10E4C05
:10B4B000B44209D1002412E062681AB1226812680D
:10B4C000AA420CD00C34F0E763680BB90C34EFE7F8
:10B4D00023682846196801F0E3FE0028F6D12046CB
:10B4E00070BD00BF78480120DC4701202DE9F34101
:10B4F0000546884600F0C8FD01224FF00003294CA4
:10B5000062F30203284A042DA4EB02046FF3C5037F
:10B5100098BF264AC4F3C90464F38F13ADF8003012
:10B5200007464FF0000394BF52F82520204A2946D1
:10B53000204801F0CDFAD8F81C30C3F308035BB102
:10B540004FF00001012363F302016FF3C50164F3BF
:10B550008F11194801F083FA4FF00006012363F3BD
:10B5600002066FF3C506384664F38F1602F0C6F97B
:10B57000B0B10278114B002A08BF1846FDF734F924
:10B580003346024639460E4801F08AFA41462846BB
:10B59000FFF7F6FE384602B0BDE8F041FEF73EBDCB
:10B5A0000648EBE7FCDC0000DCDC000064DE0000A9
:10B5B0004DE5000063E500008BE500005BE5000061
:10B5C000ACE5000008B50B4D4FF02002EFF31183FE
:10B5D00082F31188BFF36F8F02F0B7F9012104469F
:10B5E0000228D8BF084602F0C0F92C62FEF7DEF848
:10B5F000EAE700BF080301200248034A0021121AAB
:10B6000001F0AFBE000001207814012008B5064803
:10B61000064A0749121A01F077FEBDE80840054ABC
:10B620000549064801F070BEB8470120B048012026
:10B630001CE60000000000001CE6000000000120E5
:10B64000012208B50B4B02201A70FFF713FF0A4ABC
:10B650000A490B4801F08FF90320FFF70BFF00F0B8
:10B66000F1FDFCF775FF074A137B23F00103137309
:10B6700008BD00BF77140120A4DF0000C4E500006E
:10B68000E1E500009C02012080B5A2B0FDF710F8B2
:10B69000334B83F308880024E023324D012785F8DB
:10B6A0002230EC772C766C76AC766B6A2E4E43F4B7
:10B6B000E0236B62FEF78CFCFEF772F84FF0FF336D
:10B6C000AB62EB6207AB6C222146184601F049FEE3
:10B6D000B06020468DF82970FFF7CCFE3846FFF7A2
:10B6E000C9FE224D00F04EFC214B4FF48062CDE9A3
:10B6F0000473CDE902441F4BCDE900441E4928469E
:10B70000756200F035FD6B7B23F0040213F01B0F14
:10B710006A7304D1AB6913B9284600F01BFA174BC2
:10B72000012205930F23CDE903320023144DCDE907
:10B73000013300934FF4A072124B1349284600F0D6
:10B7400017FD6B7B4FF4806223F004036B730F4B88
:10B750000949C6E906330548064BF560FEF7BEF811
:10B76000B825012000ED00E0080301209C02012023
:10B770000BE6000041B600007818012010E600003A
:10B7800030020120C5B50000781C012020030120F3
:10B7900070B50E4B0E4CA34201D3002070BDD3E90F
:10B7A000030141EA000212F003020BD19D685A61C5
:10B7B000AA4201D11C33EEE75E6901320E60596185
:10B7C0000144F5E76FF01500E8E700BF7848012075
:10B7D0007848012010B513460C464FF02002EFF3D5
:10B7E000118182F31188BFF36F8F426962B12260C9
:10B7F00043691B684361836901338361002081F3DE
:10B800001188BFF36F8F0DE01BB923606FF00B0041
:10B81000F5E70246044800F031FB18B9034B9B687A
:10B820005B69236010BD00BF78140120080301206C
:10B8300070B504460D464FF02003EFF3118683F3F5
:10B840001188BFF36F8F02F021F880B100212A68C0
:10B8500081664261427BD20603D183690BB900F055
:10B8600079F93146BDE87040074801F0B7BF2B6851
:10B8700062691A602B686361A369013BA36186F367
:10B880001188BFF36F8F70BD78140120F8B504469E
:10B890000F464FF02003EFF3118583F31188BFF3B8
:10B8A0006F8FC26830495AB180688E68B04215D037
:10B8B000B7B985F31188BFF36F8F6FF00F000CE0FD
:10B8C0008B6893F90E3023618B680132E260A360CC
:10B8D00085F31188BFF36F8F0020F8BD2369F2E76D
:10B8E00090F90E3096F90E109942A8BF194621EA38
:10B8F000E17199422BDA00F003FB06463B462246F3
:10B9000029461A4800F0BAFA0028E6D04FF0200382
:10B91000EFF3118583F31188BFF36F8F23682169DB
:10B920009C4207D033B193F90E309942A8BF194613
:10B9300021EAE171A06890F90E30994209D16EB107
:10B9400029460A4801F04AFF6FF00A00C5E70026C1
:10B95000D4E700F0D5FA0028F2D1F0E785F311889A
:10B96000BFF36F8FF0E700BF0803012078140120B8
:10B9700038B583680446002B3BD0214A9268934235
:10B980003AD1DA7B013ADA73C368012B05D0013B67
:10B99000C36000F0C3F8002038BD4FF02003EFF380
:10B9A000118583F31188BFF36F8F0169806890F967
:10B9B0000E30994201D000F0A3FA204601F066FF54
:10B9C000A06080B190F90E20226100228266427B45
:10B9D000D20603D183690BB900F0BCF829460948A7
:10B9E00001F0FCFED5E7E06085F31188BFF36F8FAF
:10B9F000CFE76FF01500CFE74FF0FF30CCE700BF87
:10BA0000080301207814012010B5084C23685BB1AD
:10BA1000FDF792FD2368064A184410610021BDE835
:10BA20001040184601F0A1BF10BD00BF4003012027
:10BA300008030120F8B50D464FF02003EFF3118401
:10BA400083F31188BFF36F8F4FF4004140F2E73664
:10BA500000270022E1FB0067094B30461A61394696
:10BA60004FF47A720023FCF7E9FB064B1860064B93
:10BA70001D60FFF7C9FF84F31188BFF36F8FF8BD16
:10BA800008030120400301203C0301204FF0200364
:10BA9000EFF3118183F31188BFF36F8F044B9A6822
:10BAA000D37B013BD37381F31188BFF36F8F704752
:10BAB00008030120094B03F12802824205D19B684B
:10BAC0008B4202D14B7BDB0607D1D1E900231A6000
:10BAD0000A6853600023C1E900337047080301205E
:10BAE00038B50D4C024604F1280001F098FE0546D9
:10BAF00000B9E568A3684AB95A7BD20606D1AA699B
:10BB000022B9DA897F2A01D9636238BD9D4201D00A
:10BB1000FFF77AFF6562F8E70803012010B54FF0E0
:10BB20002003EFF3118483F31188BFF36F8F084B69
:10BB300000209A68D37B0133D373FFF7D1FF84F3DE
:10BB40001188BFF36F8FBDE8104001F05EBE00BFEB
:10BB500008030120F8B54FF02003EFF3118483F3BD
:10BB60001188BFF36F8F164A114651F8283F8B4258
:10BB70000CD05BB1D66A90F90E5093F90E70AF42BB
:10BB80000BDCB34202D01B68002BF6D1D36A0160F4
:10BB90004360D36A1860D06205E05A68C0E9003299
:10BBA0005A6810605860437B63F07F034373002042
:10BBB000FFF796FF84F31188BFF36F8FF8BD00BFC6
:10BBC00008030120F8B504464FF02003EFF3118578
:10BBD00083F31188BFF36F8F90F90D30002B03DAD8
:10BBE00001461848FFF766FF174A02F12801D2E91B
:10BBF0000A308B420BD053B194F90E6093F90E705A
:10BC0000B7420ADC834202D01B68002BF6D1C4E99C
:10BC10000010D36A1C60D46205E05968C4E90031A1
:10BC200059680C605C60637B906863F07F036373AA
:10BC3000031B58425841FFF753FF85F31188BFF3A8
:10BC40006F8FF8BD3003012008030120154A164903
:10BC500038B50C689368A342144603D1BDE8384058
:10BC6000FFF7D2BE00250D6010490968B9B1D98926
:10BC70007F2914D80E4993F90E5009688D420EDBC6
:10BC80000C498B420BD0996949B91169814203DC97
:10BC90001846FFF797FFE1E7091A116138BD002345
:10BCA0002361FBE708030120380301204003012042
:10BCB0003C0301203002012070B50446183001F029
:10BCC0002EFE4FF02003EFF3118683F31188BFF3AC
:10BCD0006F8F94F90D30002B07DA21460E48FFF7DD
:10BCE000E9FE637B03F07F0363730C4D637BA868FD
:10BCF00043F010036373031B58425841FFF7F0FEF3
:10BD000086F31188BFF36F8FAB68A34203D1BDE800
:10BD1000704001F07ABD70BD30030120080301209E
:10BD2000036D70B5044603B1984704F1180001F0A3
:10BD3000F6FD4FF02003EFF3118583F31188BFF375
:10BD40006F8F204601F018FD0646D8B194F90D30EA
:10BD5000002B07DA21461248FFF7ACFE637B03F0A5
:10BD60007F0363730F4B9868021B50425041FFF7EB
:10BD7000B7FE637B43F00803637385F31188BFF359
:10BD80006F8F70BD637B9B07F3D52146A068FFF7DB
:10BD900091FE637BA66023F002036373E9E700BFB3
:10BDA000300301200803012038B504464FF020037A
:10BDB000EFF3118583F31188BFF36F8F90F90D3086
:10BDC000002B07DA01460948FFF774FE637B03F096
:10BDD0007F036373064B9868031B58425841FFF773
:10BDE0007FFE85F31188BFF36F8F38BD30030120CC
:10BDF0000803012070B504460D461646FFF7D4FF30
:10BE0000637B43F002036373EDB12B68A5609D4231
:10BE10000CD05BB194F90E2093F90E1091420CDC1A
:10BE200069688B4202D01B68002BF5D16B682560D6
:10BE300063606B681C606C6005E05A68C4E900329E
:10BE40005A6814605C60731C15D04FF4004540F2D2
:10BE5000E730002126EAE6764FF47A72C5FB060148
:10BE60000023FCF7EBF90449421C04F11800BDE87B
:10BE7000704000F07DBA70BD2BD8000010B50C46A4
:10BE80001146064A9068064A10601A46FFF7B2FF4C
:10BE90002046BDE81040FDF7BDBC00BF08030120EF
:10BEA00038030120F8B5461C01F079FD34184FF035
:10BEB0002003EFF3118783F31188BFF36F8F0D4DCC
:10BEC0000D4BA8681860FFF76FFFA8680B49324652
:10BED000183000F04DFAAA683846537B43F010033F
:10BEE0005373FDF797FC01F05AFD201A20EAE07029
:10BEF000F8BD00BF08030120380301202BD8000043
:10BF00002DE9F84304464FF02003EFF3118983F342
:10BF10001188BFF36F8F01F02FFC4EB2804668B3DB
:10BF2000174D214605F128073846FFF7C3FDAB6AD8
:10BF3000A673BB422A460AD04BB1E96A93F90E00B8
:10BF4000B0420BDC994202D01B68002BF6D1D36AB9
:10BF500027606360D36A1C60D46205E05A68C4E954
:10BF600000325A6814605C600120FFF7B9FD89F364
:10BF70001188BFF36F8F4046BDE8F883A673F6E7DC
:10BF8000080301200021044B084603F12802C3E9FD
:10BF90000A22FFF74FBD00BF08030120F8B5244C6B
:10BFA000244BA2689A4236D04FF02003EFF311865B
:10BFB00083F31188BFF36F8F04F12805A168284629
:10BFC000FFF778FDA26AA368AA420CD05AB1E06AD2
:10BFD00093F90E1092F90E708F420BDC824202D060
:10BFE0001268002AF6D1E26A1D605A60E26A1360A4
:10BFF000E36205E05168C3E9002151680B605360BA
:10C000005A7B012062F07F025A73FFF769FD86F3C5
:10C010001188BFF36F8F4FF02003EFF3118083F38C
:10C020001188BFF36F8FBDE8F840FDF7F3BB00BF89
:10C03000080301203002012038B5431C044605D115
:10C04000104B986800F0DEF8204638BD4FF40045EC
:10C0500040F2E73000214FF47A72E5FB040100233F
:10C06000FCF7ECF8044648B9FFF798FF4FF47A70F4
:10C0700084FB0001C40B44EA4140E6E7FFF712FFEE
:10C080000446F3E708030120014B9868704700BF9E
:10C090000803012070B504464FF02003EFF311862A
:10C0A00083F31188BFF36F8F01F0F0FB054670B189
:10C0B000437BDB0603D183690BB9FFF74BFD0023FC
:10C0C000AB663146BDE87040044801F087BBD4E957
:10C0D00002329A4218BF0133A360F2E778140120BC
:10C0E00010B402460B464FF02000EFF3118180F3AD
:10C0F0001188BFF36F8F946844B1013C946081F361
:10C100001188BFF36F8F002010BC704733B981F3E3
:10C110001188BFF36F8F6FF00F00F5E7014810BC77
:10C12000FFF7ACBE7814012010B54FF02002EFF3FA
:10C13000118482F31188BFF36F8F427B510704D4BF
:10C1400084F31188BFF36F8F10BD22F0040112F049
:10C150001B0F417303D183690BB9FFF7FBFC214629
:10C16000BDE81040014801F039BB00BF7814012040
:10C1700030B587B00E9D044604950D9D03950C9D2A
:10C1800002950B9D01950A9D0095FDF785FB044BDB
:10C190009B6813B9236607B030BD1B6EFAE700BF7A
:10C1A0000803012070B5002686B005960E9E0F9DEF
:10C1B00004960D9E044603960C9E02960B9E0196D5
:10C1C0000A9E0096FFF7D4FF6B1C03D02DB92046C2
:10C1D000FFF7AAFF204606B070BD4FF4004640F2BC
:10C1E000E73000214FF47A720023E6FB0501FCF7EB
:10C1F00025F80349421C04F1180000F0B9F8E9E7FA
:10C200002BD8000038B505464FF02003EFF311841A
:10C2100083F31188BFF36F8FFFF74EFD074B9B68C9
:10C22000AB4205D12146BDE83840054801F0D6BAF9
:10C2300084F31188BFF36F8F38BD00BF080301205E
:10C24000781401202DE9F04F284E294DB04687B0D3
:10C25000B54205F1300410D3FFF718FC4FF4004944
:10C2600040F2E7360027224CDFF888A0444521D36E
:10C2700007B0BDE8F04FFFF751BC54F8043C0593FC
:10C2800054F8103C049354F8143C039354F8183CAD
:10C29000029354F81C3C019354F8203C009354E959
:10C2A0000A2354E90C01FFF763FF54F8303CDD64C6
:10C2B0002546CDE7616A4B1C04D0256821B9284684
:10C2C000FFF732FF3034D1E7B346BC46E9FB01BC8F
:10C2D0004FF47A72002358466146FBF7AFFF514690
:10C2E000421C05F1180000F043F8EBE77848012004
:10C2F000784801202BD80000034B1B680BB9FDF7D1
:10C300001BB90020704700BF44030120036840B1FF
:10C31000084A5268904204D01BB19A6881680A4466
:10C320009A604268136003685A600023C0E90033D2
:10C33000704700BFD44701200B4B10B51C689C42CE
:10C3400008BF0024FFF7D8FF54B1A368181A20EAE9
:10C35000E070064B1B6913B19842A8BF184610BD88
:10C360006FF00040F5E700BFD4470120080301202B
:10C3700070B504461646C1604FF02003EFF31185F7
:10C3800083F31188BFF36F8FFFF7B6FF012EACBFA9
:10C3900080190130174BA0601A689A4201D05E687C
:10C3A00032B95A68236062605A6814605C600BE0BE
:10C3B0009068A168884216DD411A91605168C4E90D
:10C3C000002151680C6054601A689A4206D0944269
:10C3D00004D1FFF7B1FF0021FDF756F885F311886E
:10C3E000BFF36F8F70BD091A9642A160D9D0126851
:10C3F000D6E700BFD44701202DE9F04B0446FFF7F4
:10C4000025FC4FF02003EFF3118583F31188BFF370
:10C410006F8F214F214EB846DFF884903460D9F8F1
:10C42000004032684C45D7E900BC05D024B1A36870
:10C43000934214DD9B1AA36000241BEB02004CEB1B
:10C44000E271C8E900013460FFF776FF2146FDF78D
:10C450001BF885F31188BFF36F8FBDE8F08B1BEBE2
:10C4600003004CEBE371D31A33600023C7E90001EA
:10C47000A3602046FFF74AFF85F31188BFF36F8F53
:10C48000E36898474FF02003EFF3118583F3118899
:10C49000BFF36F8FC3E700BF0000012044030120FA
:10C4A000D44701202DE918484FF02003EFF3118401
:10C4B00083F31188BFF36F8FFDF73EF8074BD3E985
:10C4C000002312EB000B43F1000C5846614684F345
:10C4D0001188BFF36F8FBDE8188800BF00000120EE
:10C4E000026A38B5002A044602DD0E49FFF740FF14
:10C4F000636A01336362A3690BB12046984754F81D
:10C50000105FA5420DD065B1284601F04EF96B7B56
:10C51000DB0604D1AB6913B92846FFF71BFB0023E8
:10C52000AB6638BDE1C400002DE9F34140F2E736C7
:10C530000027044688464FF400453046394600231C
:10C54000E5FB02014FF47A72FBF778FE3946009062
:10C5500030464FF47A720023E5FB0801FBF76EFECC
:10C560000190204601F0DBF9009B20462362002366
:10C57000019A0349636202B0BDE8F041FFF7F8BEDB
:10C58000E1C4000038B5074C074DAC4201D3002090
:10C5900038BD04F114032046C4E9053300F006F861
:10C5A0001C34F2E77848012078480120FF232DE968
:10C5B000F74F4568002229464FF00C0A4FF0200B38
:10C5C0000789046805FB07FCC372837A64440193FE
:10C5D000019B934208DC002319468F4205EB030CB4
:10C5E00021DC03B0BDE8F08FBCFBF1F3202B84BF4E
:10C5F0001F3393FBFBF30AFB02FED0F80C804FEADB
:10C60000910108EB0E0606F10409C6E9019921F033
:10C61000030194BFC27248F80E4002F1010288BFC4
:10C6200004EB8304D4E7C268066802F1040EF41830
:10C6300046F803E093680131636093681C6094607E
:10C640006346CAE70020704770B50D460446452092
:10C65000A04729465220A04729462346BDE87040FE
:10C660005220184730B58A680C68551C14B14B68C5
:10C67000934201DC8D6030BD013B934208BF002234
:10C680008D600CBFE254A054F5E72DE9F04F002770
:10C6900005460E4692461C464FF0FF39B846BB464B
:10C6A00089B09AF8000010B909B0BDE8F08FBBF16D
:10C6B000000F07D1252800F04E813146A8470AF126
:10C6C000010AEEE7642868D01AD839280BD8312837
:10C6D0005AD22D2800F04681302846D0252808D18E
:10C6E0003146A8477AE0582800F0B480632800F06B
:10C6F0002C8131462520A84731469AF80000F0E702
:10C70000702800F09D800DD8692846D06C2803D190
:10C710006C2F26D14C27D2E76828EAD1682F20D188
:10C720004827CCE7752870D017D87328E1D1226844
:10C7300004F1040B11460C4614F8010B002840F0DC
:10C74000F980B8F1030F40F013818C1AA9EB0404AF
:10C75000002C00F3F5805C4640E078287AD07A28F7
:10C76000C7D1002FC5D10746A9E7B9F1000F0EDAEE
:10C77000B8F1000F00F0F980A0F13009B8F1000F16
:10C7800008BF4FF002089AE7B9F1000FF4DB0A2264
:10C7900002FB0909A9F13009F0E77A2F03D1D4F897
:10C7A00000B004341EE06C2FF9D04C2FF7D14FF0BD
:10C7B000000C4FF0FF3B073424F0070303F108049B
:10C7C000D3E9002312F1004043F100018C4508BF7A
:10C7D000834506D231462846FFF736FF4FF0000B5F
:10C7E0006DE79346BBF1000F06DA31462D20A847CE
:10C7F000CBF1000B09F1FF3943465A46CDF80090C2
:10C8000031462846FBF7ACFEE8E77A2F02D12268D2
:10C81000043411E06C2FFAD04C2FF8D100214FF0E6
:10C82000FF30073424F0070303F10804D3E90023A1
:10C83000994208BF9042CDD3CDF800904346DFE740
:10C8400031463020A84731467820A8474FF00809E4
:10C850004FF001089AF80020702A05D123680434AB
:10C860000493002302930CE06C2FF7D04C2FF5D1EA
:10C87000073424F00702136802F108040493536894
:10C88000029300221023039205924022043A029957
:10C890000498C2F1200CA2F1200ED04001FA0CFC49
:10C8A00040EA0C0021FA0EFE40EA0E0010F00F00E4
:10C8B00008D1059901B942BB4FF0300C08E0CDF822
:10C8C00014B0E3E709288CBF4FF0570C4FF0300C41
:10C8D00031466044CDE90523A847039B0133039308
:10C8E000DDE90523002AEAD1B8F1030F7FF476AF22
:10C8F000039BC3EB490BBBF1000F7FF76FAF3146D2
:10C900002020A8470BF1FF3BF5E7591E99450691FA
:10C9100007DBB8F1010F06D1314630200792A84756
:10C92000079A069BB2E7B8F1020FFAD10792314697
:10C930002020F4E731460292A8472146029AFAE6FF
:10C9400031462020A847013C02E73146206804F127
:10C95000040BA847FFE65F46D8464FF0FF394FF07B
:10C96000010BACE64FF00308A9E64FF00108A6E67C
:10C970005C468346A3E60FB407B504A951F8040B3F
:10C98000019100F0C0F803B05DF804EB04B070470B
:10C99000044608B5084611461A46A047FFF774FB3F
:10C9A000FDF73CFB70474FF02003EFF3118183F359
:10C9B0001188BFF36F8F4FF040230122C3F8042783
:10C9C000C3F80429C3F8002B81F31188BFF36F8FDC
:10C9D0000020704700F0B1BE0023C0E9003370476B
:10C9E000036823B90160002341600B60704743680E
:10C9F0001960F8E70068704703680BB11A680260B5
:10CA00001846704708B5FCF7ADF818B1012343602C
:10CA10000023038108BDFCF7A9BD00207047002357
:10CA2000F0B51A461C46012710F8015B0DB18A4289
:10CA300001D31846F0BD252D02D184F00104F3E79F
:10CA4000002CF1D045F02006613E192EECD8732D54
:10CA500004BF07FA02F4234301320024E4E738B5A7
:10CA600005460C46FFF7CEFF28B105612146BDE81B
:10CA70003840FBF7E5BF38BD70B504460E46154695
:10CA8000FFF7C0FF58B101220461447A466162F3A6
:10CA9000071444722946BDE87040FBF7D1BF70BD52
:10CAA0002DE9F0410546884617461E46FFF7AAFFC6
:10CAB00060B102230561457AC0E9058763F3071574
:10CAC00045723146BDE8F041FBF7BABFBDE8F081E1
:10CAD0002DE9F8430546894690461F46BDF820607B
:10CAE000FFF790FF68B103230561457AC0E9059817
:10CAF00063F307154572C7613146BDE8F843FBF79C
:10CB00009FBFBDE8F88300B5C3B002460B4601A83D
:10CB100040F20111FBF776FD40F20112824228BF7C
:10CB2000024601A9002000F094F818B14FF000016E
:10CB3000FBF786FF43B05DF804FB2DE9F8431C4684
:10CB400003890E469B08A3429DF8207003D800235A
:10CB50001360BDE8F88311682144994284BF191B12
:10CB600011600C2BD2F8009028D9072CD0F8148033
:10CB70002BD8082318304B4528BF4B4620441D4670
:10CB80001A46FFB1314600F0BFFBA9EB05092E4460
:10CB9000B9F1000FDDD0C4F11C054D4528BF4D464D
:10CBA000201D40442A46BFB1314600F0ADFBA9EB41
:10CBB0000509D8F800802E440024E9E714304FF02E
:10CBC0000008D8E701463046DDE7083C1B2CDFD9DA
:10CBD000D8F800801C3CF9E701463046E5E7043010
:10CBE000D0E8EF3F0133C0E8E23F002AF8D17047B8
:10CBF000407A00097047437A1B098B4216D9032BF0
:10CC000003D800EB810148697047012903D800EB84
:10CC100081018869704743690239062903D803EB0B
:10CC200081014868704707391B68F6E700207047A4
:10CC30000346021DD2E8EF1F0139C2E8EC1FBCF128
:10CC4000000FF7D15B680BB9FBF79EBF7047006917
:10CC500070472DE9F84343F6FF75954280460E462E
:10CC6000174628BF1546FBF77DFF044680B3012316
:10CC70004360037A0C2F43F0010303720389C0F869
:10CC8000108065F38F03038100F1140817D908227F
:10CC90003146183000F038FB00239946227A636150
:10CCA00042F0020222720836083D8DB1FBF75AFFAE
:10CCB000074680B92046FBF767FF3C4608E02A4656
:10CCC0003146404600F020FB237A6FF34103237284
:10CCD0002046BDE8F8831C2D2F4628BF1C27C8F826
:10CCE00000003146C0F8009080463A46043000F01B
:10CCF0000BFB3E44ED1BD8E713B500240094FFF76F
:10CD00001CFF02B010BDF8B506460D4614461F467E
:10CD1000214628463A46B047241A0544F8D1F8BDC2
:10CD20002DE9F0478EB00EAF81460D46FFF78FFF1D
:10CD300006464846FFF75CFF4FF000088246830036
:10CD40000E3323F00703ADEB030D0EACD04516D127
:10CD50004846FFF74DFF0F281ED8DFE810F01900F6
:10CD6000200026002D00360041004E005D006E00C0
:10CD700081009600AD00C600E100FE001D014146A5
:10CD80004846FFF738FF44F8280008F10108DDE7BE
:10CD900031462846FBF73CFFBD46BDE8F0872268D8
:10CDA00031462846FBF734FFF6E7D4E90023314645
:10CDB0002846FBF72DFFEFE7A36831460093D4E93F
:10CDC00000232846FBF724FFE6E7E368314601939A
:10CDD000A36828460093D4E90023FBF719FFDBE79B
:10CDE000236931460293E36828460193A3680093C0
:10CDF000D4E90023FBF70CFFCEE7636931460393C8
:10CE0000236928460293E3680193A3680093D4E959
:10CE10000023FBF7FDFEBFE7A36931460493636976
:10CE20002846039323690293E3680193A368009360
:10CE3000D4E90023FBF7ECFEAEE7E3693146059346
:10CE4000A369284604936369039323690293E36803
:10CE50000193A3680093D4E90023FBF7D9FE9BE775
:10CE6000236A31460693E36928460593A369049330
:10CE70006369039323690293E3680193A3680093B2
:10CE8000D4E90023FBF7C4FE86E7636A31460793C3
:10CE9000236A28460693E3690593A36904936369AB
:10CEA000039323690293E3680193A3680093D4E991
:10CEB0000023FBF7ADFE6FE7A36A31460893636A70
:10CEC00028460793236A0693E3690593A3690493AD
:10CED0006369039323690293E3680193A368009352
:10CEE000D4E90023FBF794FE56E7E36A3146099341
:10CEF000A36A28460893636A0793236A0693E36943
:10CF00000593A36904936369039323690293E36818
:10CF10000193A3680093D4E90023FBF779FE3BE774
:10CF2000236B31460A93E36A28460993A36A089360
:10CF3000636A0793236A0693E3690593A3690493DD
:10CF40006369039323690293E3680193A3680093E1
:10CF5000D4E90023FBF75CFE1EE7636B31460B93BD
:10CF6000236B28460A93E36A0993A36A0893636ACA
:10CF70000793236A0693E3690593A369049363699E
:10CF8000039323690293E3680193A3680093D4E9B0
:10CF90000023FBF73DFEFFE6A36B31460C93636B6A
:10CFA00028460B93236B0A93E36A0993A36A0893B9
:10CFB000636A0793236A0693E3690593A36904935D
:10CFC0006369039323690293E3680193A368009361
:10CFD000D4E90023FBF71CFEDEE6426810B5D2E977
:10CFE0000023044681680068FFF78DFE0022636815
:10CFF0001A6010BD38B54B6805461A68CB680C46F8
:10D000009A4202D10846FFF7E8FF6368D3E8EF2FA2
:10D01000511CC3E8E01F0028F8D1A36800209D54EC
:10D0200038BD0C228368C9B202FB01314B7A23B9A7
:10D03000087AB0FA80F04009704702207047026811
:10D040002DE9F041D2F80880CCB287684FF0200378
:10D05000EFF3118683F31188BFF36F8F0C226243C5
:10D06000B9180B7A43B3013BDBB20B723BBB250112
:10D07000BB504B6008EB05035B68CBB9012245440C
:10D08000EB7A03F1804303F5A0431A6000222B8959
:10D0900003F1804303F5A0431A600C21002001FB3B
:10D0A0000474607286F31188BFF36F8FBDE8F0815E
:10D0B00098470028E2D1F0E76FF04400F2E7002043
:10D0C000F0E738B50C248368054604FB01340123DE
:10D0D00063724FF02003EFF3118183F31188BFF3E4
:10D0E0006F8F23682BB160681A688342226008BF83
:10D0F000626081F31188BFF36F8F03B938BDD3E944
:10D10000012128469047E4E70022FCF7AFB87047BA
:10D1100070470369C1688B4297BF826803F1FF3390
:10D12000D21802F1FF3294BF501A581A70472DE9F5
:10D13000F041D0E902670446F61B406896428846F3
:10D140001546384405D900F0DFF83D44E560BDE8F8
:10D15000F0813246AD1B00F0D7F82A4608EB0601F5
:10D16000606800F0D1F8F1E72DE9F84306468946FA
:10D1700017464FF00008C5683469B368A54228BF58
:10D18000E418013C621B5C1BBC4228BF3C46944235
:10D1900028BF1446706849462844224600F0B4F877
:10D1A000B3682544AB4208BF00253F1BA044A144FF
:10D1B000F560E1D14046BDE8F883FCF7F1B908B568
:10D1C000FFF7FBFF002008BDFCF7F6BA0146006838
:10D1D000FCF7A2BB08B5FCF7F9FABDE80840FCF77C
:10D1E00097BA07B5002101A8FDF702F903B05DF871
:10D1F00004FB30B54B6885B00C689DF808200D899C
:10D200000094498924F01F04013B234465F3040280
:10D2100061F3471223F01F030F288DF808200393B2
:10D22000044605D9FCF762FF0446204605B030BD30
:10D230006946FCF743FFF8E740E800F313F4803F4A
:10D24000D8B208BF6FF0150070470346013911F8D6
:10D25000012F0AB91A70704703F8012BF7E770B570
:10D26000054601392C4642B111F8013F561E2BB933
:10D270002A4404F8013BA242FBD170BD05F8013BF2
:10D280003246EFE7C9B2027803468A4200F1010054
:10D2900004D0002AF7D1002918BF00231846704790
:10D2A0000138013910F8013F11F8012F934202D1E2
:10D2B000002BF7D11A46981A704710B55AB10139A8
:10D2C000841810F8012B11F8013FA04201D09A42B6
:10D2D000F7D0D01A10BD1046FCE7431A934210B5A0
:10D2E00000EB020308D3024601399A420BD011F831
:10D2F000014F02F8014BF8E70A4412F8014D8A4247
:10D3000003F8014DF9D110BDF0B581EA0004A5077D
:10D3100003460BD0013B0A4491421DD1F0BD002AC7
:10D32000FCD011F8014B013A03F8014B9C07F6D1F0
:10D330000C461D1F8F183E1B032E08D86FF00305E7
:10D34000940805FB0422A40023442144E2E754F896
:10D35000046B45F8046FEEE711F8014B03F8014F39
:10D36000DAE70346F0B5C9B29C070FD11D4641EA82
:10D37000012444EA04449F187E1B032E0CD8940811
:10D3800003EB840413449C4209D1F0BD002AFCD075
:10D3900003F8011B013AE7E745F8044BECE704F812
:10D3A000011BF0E7034670B5B1FBF2F602FB161164
:10D3B00009298CBF272500251C463031294404F853
:10D3C000011B31462EB95E70241A834203D82046D1
:10D3D00070BD2346E8E71A78017803F8011900F8D0
:10D3E000012BF2E7D0E900232DE930485FEA530C26
:10D3F0004FEA320B002502F001041BEB04024CEB58
:10D400000503C0E90023BDE830880521D0E90023E9
:10D410002DE9F04F12F1020843F10009B9FBF1F5D3
:10D42000002601FB05F7B8EB060869EB07094FEA90
:10D43000D80646EA4976B6FBF1FC0024C2464FEA1C
:10D44000CC06A6FB0189A2194FEA5C7745EB0703DE
:10D450001446BAEB0802B2FBF1F21D46A41845F1DE
:10D460000005C0E90045BDE8F08F0B682DE91048C4
:10D47000002B13DD013B0B600A2102684468A2FB0C
:10D4800001BC5A4601FB04CC2CF07043C0E90023D8
:10D490004FEA1C7130310846BDE810883021FAE7A8
:10D4A0004FF0FF3070474B68012B07DD0B68187099
:10D4B0000B6801330B604B68013B4B6000207047E9
:10D4C00010B504688068A46801292468C06903D184
:10D4D00058406060002010BD00334FF0010118BFBC
:10D4E0000123D04000F001009140834214BFA160AD
:10D4F000E160EFE770B504688068A468C0692568DA
:10D5000001296E692C696D6880EA040084EA0504CB
:10D5100004EA060480EA04001CBFD04000F00100C9
:10D520001860002070BD836830B5186858B10024B9
:10D53000814213D108685CB95C681860A14200D1CF
:10D5400058600020086072B9002030BD2846EFE71F
:10D5500020605868814208BF5C60F2E705680446B5
:10D56000002DF3D13AB11A680A6058681960002892
:10D57000EAD15960E9E76FF01500E6E7F8B585688C
:10D580000F462968064669B10C68EB688A683B401B
:10D59000134203D04B683A463046984714B12146AF
:10D5A0002468F2E7F8BD01292DE9F04118BFD4B293
:10D5B000064612BF25461F2500244FF00108876844
:10D5C000AC4202D90020BDE8F081FB6808FA04F201
:10D5D00023EA0203FB6021463046FDF74BFC00289E
:10D5E000F1D10134E4B2EBE7F8B501250026026879
:10D5F00083689768D3E902120A40D3E90510014312
:10D6000022EA01023968DC691B6909695C404C4007
:10D6100022EA04040AB92046F8BD2A4209D03B791F
:10D6200006F01F00002140EA4310FDF70DFC22EA3E
:10D63000050201366D00EDE7F8B501270026846884
:10D6400003689D68D4E902321A40D4E905310B43DE
:10D6500022EA030202B9F8BD174212D0E169236938
:10D6600095F804C04B40F34013F0010F06F01F0083
:10D6700014BF0221032140EA4C10FDF7E5FB22EA2A
:10D68000070201367F00E5E701292DE9F04118BFC7
:10D69000D4B2064612BF25461F2500244FF00108CC
:10D6A0008768AC4202D90020BDE8F081FB6808FA27
:10D6B00004F21343FB6021463046FDF7DBFB0028F4
:10D6C000F2D10134E4B2ECE70B46826892E8030041
:10D6D00083E803000020704703689B681B68D3F849
:10D6E0008004C3F880047047036882689B681B68E5
:10D6F000D3F8100138B1127A00200A700122C3F861
:10D7000010011A6070474FF0FF30704782B002AAD4
:10D7100002F8011D002103689B681B68C3F82011F3
:10D72000C3F844250122C3F848259A60D3F8201194
:10D730000029FBD0DA6002B07047FDF78BBEFFF71F
:10D74000E7BC30B50024846141EA020414F003040C
:10D75000C0E9023201610CD14461A34203D1C0E9A6
:10D760000000002030BD456901340D604161114465
:10D77000F3E76FF01500F5E7437BDB0603BF806935
:10D78000B0FA80F040090020704710B54FF0200338
:10D79000EFF3118483F31188BFF36F8F00F03FF82C
:10D7A00084F31188BFF36F8F10BD38B504464FF076
:10D7B0002003EFF3118583F31188BFF36F8F0146C8
:10D7C0008068FEF777F9637B23F00203637385F3C8
:10D7D0001188BFF36F8F0023A36038BD21B9EFF329
:10D7E000058008B9FCF716B881F31188BFF36F8F75
:10D7F0007047034620B9EFF305820AB9FCF70AB86F
:10D8000083F31188BFF36F8F70474FF02003EFF35E
:10D81000118083F31188BFF36F8FFFF7EABF0368AE
:10D82000984214BF18460020704750F8103C70B55D
:10D830000446A0F11805CBB14FF02003EFF3118699
:10D8400083F31188BFF36F8F294650F8100CFEF751
:10D8500031F914F80B3C23F0020304F80B3C86F377
:10D860001188BFF36F8F002344F8103C14F80B3C71
:10D87000284623F0140304F80B3CFFF77DFF20B18A
:10D880002846BDE87040FEF765B970BD38B54FF069
:10D890002003EFF3118283F31188BFF36F8FFFF73B
:10D8A000BEFF044682F31188BFF36F8FC8B14FF0FB
:10D8B0002003EFF3118583F31188BFF36F8F0146C7
:10D8C0008068FEF7F7F8637B23F00203637385F348
:10D8D0001188BFF36F8F002304F11800A36000F0DC
:10D8E0001EF8204638BDEFF30580003018BF012038
:10D8F0007047FAF79BBE6FF04600704700207047F4
:10D9000010B5029C8373047300230424C37344730F
:10D91000C0E90633C0E91333C0E9161210BD10B5D3
:10D920004FF02002EFF3118482F31188BFF36F8F61
:10D9300003683BB1FEF7EAFC002084F31188BFF3D3
:10D940006F8F10BD6FF01500F7E710B54FF0200393
:10D95000EFF3118483F31188BFF36F8FFEF7ECFCB4
:10D9600084F31188BFF36F8F10BD70B504460E4667
:10D970004FF02003EFF3118583F31188BFF36F8F0E
:10D98000FEF7DAFC012805DDA04203DD3146204622
:10D99000FBF77AFD85F31188BFF36F8F70BD08B573
:10D9A000FEF780FD08BD0023C0E9061200F1100259
:10D9B0004362C0E90422C0E900338362704710B5B6
:10D9C0000446FFF7ACFF00BBE3690BB12046984764
:10D9D00004F110000021FFF7D8FE0446A8B1FFF7BC
:10D9E000E4FE637BDB0604D1A36913B92046FEF78E
:10D9F000B1F84FF02003EFF3118083F31188BFF3E8
:10DA00006F8FBDE81040FFF7F4BE10BD7047FFFFF9
:10DA10005CA8FF7F0100000000000000C9D10000E9
:10DA200000000000C9D1000000000000C9D10000C2
:10DA300000000000C9D1000000000000C9D10000B2
:10DA4000000000008993000000000000C9D1000020
:10DA500000000000C9D1000000000000C9D1000092
:10DA600000000000C9D1000000000000C9D1000082
:10DA700000000000C9D1000000000000C9D1000072
:10DA800000000000C9D1000000000000C9D1000062
:10DA900000000000C9D1000000000000C9D1000052
:10DAA00000000000C9D1000000000000C9D1000042
:10DAB00000000000C9D1000000000000C9D1000032
:10DAC00000000000DD93000000000000C9D100004C
:10DAD00000000000C9D1000000000000C9D1000012
:10DAE00000000000C9D1000000000000C9D1000002
:10DAF00000000000C9D1000000000000C9D10000F2
:10DB000000000000C9D1000000000000C9D10000E1
:10DB100000000000C9D1000000000000C9D10000D1
:10DB200000000000C9D1000000000000C9D10000C1
:10DB300000000000C9D1000000000000C9D10000B1
:10DB400000000000C9D1000000000000C9D10000A1
:10DB500000000000C9D1000000000000C9D1000091
:10DB600000000000C9D1000000000000C9D1000081
:10DB700000000000C9D1000000000000C9D1000071
:10DB800000000000C9D1000000000000C9D1000061
:10DB900000000000DDB0000000000000C9D100005E
:10DBA00000000000C9D1000000000000C9D1000041
:10DBB00000000000C9D1000000000000C9D1000031
:10DBC00000000000C9D1000000000000C9D1000021
:10DBD00000000000C9D1000000000000C9D1000011
:10DBE00000000000C9D1000000000000C9D1000001
:10DBF00000000000C9D1000000000000C9D10000F1
:10DC000000000000C9D1000000000000C9D10000E0
:10DC100000000000C9D1000000000000C9D10000D0
:10DC200000000000C9D1000000000000C9D10000C0
:10DC300000000000C9D1000000000000C9D10000B0
:10DC4000A4DF0000A7C9000000000000A4DF00005E
:10DC50005D86000000000000A4DF0000ED910000E0
:10DC600000000000BBDF000051930000BCDD00009D
:10DC7000DBDF00001D94000000000000A4DF0000B6
:10DC8000BFD1000000000000A4DF0000EDA20000F2
:10DC90000000000065E4000019AE000028DE00006E
:10DCA0006CE4000019AE000020DE000073E4000008
:10DCB00015B3000044DE0000A4DF0000B9B300008B
:10DCC00000000000A4DF000091B700000000000089
:10DCD000A4DF000085C5000000000000CDDF0000CB
:10DCE000030000009BE4000003000000C9DE000008
:10DCF00002000000DCE300000300000008E6000072
:10DD000003000000B5DF000003000000A3DE0000F8
:10DD1000030000007AE400000100000080DD000044
:10DD2000F8000120A5DF000001000000FFFFFFFF59
:10DD3000DEE61E28EAAC45B802350000DEE61E2805
:10DD40004CBBCE8F02350000000000000000000038
:10DD50000338FDD870470000000000006DDF0000B0
:10DD600075DF00000000000000000000000000005F
:10DD70007DDF000081DF000085DF000089DF00001B
:10DD80001990000000000000000000000D9000004D
:10DD9000F58F0000D98F0000559000000C01012084
:10DDA0004A0301200100000009D100003FD000001B
:10DDB0006D9200000000000023D000000000000071
:10DDC0000000000000010004C1DF000000000000AE
:10DDD000000000000401080CC7DF00000200000082
:10DDE000E4DD00000000000056E400000600000032
:10DDF000E0FF0F00000001205EE4000021000000B1
:10DE0000E0FF0620ADAF0000C1D40000F5D4000053
:10DE100027D5000089D60000A7D50000000000002B
:10DE2000002584400000000000288440010000001C
:10DE3000E9D600000DD70000D9D600008DB1000052
:10DE4000C9D600000080004001000000DC4701202E
:10DE50003C480120484801207848012078480120AA
:10DE6000F5FFFFFF03E5000011E5000025E50000D8
:10DE700034E5000040E500006E7266353334305FF3
:10DE8000646B5F6E7266353334305F6370756170DA
:10DE9000700048656C6C6F20576F726C6421202590
:10DEA000730A00736F63006C6F6767696E67003C8D
:10DEB0006C6F675F73747264757020616C6C6F63F4
:10DEC000206661696C65643E006C6F670061726713
:10DED000756D656E7420256420696E206C6F6720F7
:10DEE0006D6573736167652022257322206D6973E8
:10DEF00073696E67206C6F675F73747264757028E6
:10DF0000292E00253032782000202020007C00259A
:10DF100063000D00206D6573736167657320647223
:10DF20006F70706564202D2D2D0D0A002D2D2D2074
:10DF3000001B5B306D0025732E0025733A20005BBB
:10DF40002530386C755D20005B253032643A253011
:10DF500032643A253032642E253033642C25303338
:10DF6000645D20002573003C25733E20001B5B315F
:10DF70003B33316D001B5B313B33336D0065727297
:10DF80000077726E00696E6600646267006D65738B
:10DF900073616765732064726F707065643A2020E6
:10DFA00020200D0A006C6F675F6261636B656E64B1
:10DFB0005F72747400706F77657200434C4F434B0F
:10DFC000006866636C6B006C66636C6B00636C6FFF
:10DFD000636B5F636F6E74726F6C007379735F63F2
:10DFE0006C6F636B005465726D696E616C005254A6
:10DFF00054005345474745520072302F61313A2053
:10E0000020307825303878202072312F61323A2044
:10E0100020307825303878202072322F61333A2032
:10E02000203078253038780072332F61343A202040
:10E03000307825303878207231322F69703A2020BC
:10E04000307825303878207231342F6C723A2020A5
:10E050003078253038780020787073723A2020307C
:10E060007825303878004661756C74696E67206970
:10E070006E737472756374696F6E20616464726527
:10E08000737320287231352F7063293A2030782538
:10E09000303878002A2A2A2A2A204255532046411D
:10E0A000554C54202A2A2A2A2A00202053746163BE
:10E0B0006B696E67206572726F7200202050726506
:10E0C0006369736520646174612062757320657291
:10E0D000726F720020204246415220416464726592
:10E0E00073733A2030782578002020496D7072656E
:10E0F0006369736520646174612062757320657261
:10E10000726F72002020496E737472756374696F48
:10E110006E20627573206572726F72002A2A2A2A35
:10E120002A204D5055204641554C54202A2A2A2A4F
:10E130002A002020537461636B696E6720657272D8
:10E140006F722028636F6E746578742061726561E8
:10E15000206D69676874206265206E6F7420766137
:10E160006C696429002020556E737461636B696E5D
:10E1700067206572726F72002020446174612041D3
:10E1800063636573732056696F6C6174696F6E00A9
:10E1900020204D4D46415220416464726573733AAC
:10E1A0002030782578002020496E7374727563746E
:10E1B000696F6E204163636573732056696F6C618C
:10E1C00074696F6E002020466C6F6174696E672DF4
:10E1D000706F696E74206C617A79207374617465F4
:10E1E00020707265736572766174696F6E206572F6
:10E1F000726F72002A2A2A2A2A2055534147452045
:10E200004641554C54202A2A2A2A2A0020204469B3
:10E21000766973696F6E206279207A65726F00206B
:10E2200020556E616C69676E6564206D656D6F72F7
:10E230007920616363657373002020537461636B9D
:10E24000206F766572666C6F772028636F6E7465D9
:10E2500078742061726561206E6F742076616C69DC
:10E2600064290020204E6F20636F70726F636573A6
:10E27000736F7220696E737472756374696F6E73F5
:10E28000002020496C6C6567616C206C6F616420B4
:10E290006F66204558435F52455455524E20696E73
:10E2A000746F205043002020496C6C6567616C20BE
:10E2B000757365206F662074686520455053520061
:10E2C0002020417474656D707420746F20657865CA
:10E2D0006375746520756E646566696E6564206932
:10E2E0006E737472756374696F6E004578636570E0
:10E2F00074696F6E206F6363757272656420696EF6
:10E3000020536563757265205374617465002A2A11
:10E310002A2A2A2048415244204641554C54202A5A
:10E320002A2A2A2A002020427573206661756C749F
:10E33000206F6E20766563746F72207461626C6505
:10E3400020726561640020204661756C74206573DD
:10E3500063616C6174696F6E202873656520626506
:10E360006C6F7729002A2A2A2A2A20446562756759
:10E37000206D6F6E69746F72206578636570746963
:10E380006F6E20286E6F7420696D706C656D656EA0
:10E3900074656429202A2A2A2A2A00526573657224
:10E3A00076656420457863657074696F6E20280017
:10E3B00053707572696F757320696E7465727275CA
:10E3C0007074202849525120002A2A2A2A2A2025FE
:10E3D0007320256429202A2A2A2A2A006D707500B4
:10E3E000506172746974696F6E2025753A2073618B
:10E3F0006E69747920636865636B206661696C651A
:10E40000642E00496E76616C696420756E64657275
:10E410006C79696E6720726567696F6E20696E64DA
:10E420006578202575004661696C656420746F20ED
:10E43000616C6C6F63617465206E6577204D50551B
:10E4400020726567696F6E2025750A002D2B2023C9
:10E450003000686C7A00464C4153485F300053529C
:10E46000414D5F30004750494F5F31004750494FA1
:10E470005F3000554152545F3000756172745F6EB9
:10E480007266785F75617274650052657365747445
:10E49000696E672073797374656D00666174616C71
:10E4A0005F6572726F72004552524F523A2043615B
:10E4B0006E6E6F742066756C66696C6C204558547E
:10E4C0005F41504920726571756573742E0D0A00A5
:10E4D0005741524E494E473A204F7074696F6E61F2
:10E4E0006C204558545F41504920726571756573C1
:10E4F00074206E6F742066756C66696C6C65642E32
:10E500000D0A0043505520657863657074696F6E1D
:10E5100000556E68616E646C656420696E74657226
:10E520007275707400537461636B206F76657266E8
:10E530006C6F77004B65726E656C206F6F70730047
:10E540004B65726E656C2070616E696300556E6B11
:10E550006E6F776E206572726F7200756E6B6E6F84
:10E56000776E003E3E3E205A455048595220464163
:10E5700054414C204552524F522025643A20257375
:10E58000206F6E20435055202564004661756C74E1
:10E5900020647572696E6720696E74657272757039
:10E5A000742068616E646C696E670A0043757272EC
:10E5B000656E74207468726561643A202570202845
:10E5C0002573290076322E312E39392D6E63733141
:10E5D0002D332D67376464616236363462303462BD
:10E5E000002A2A2A20426F6F74696E67205A65706C
:10E5F000687972204F53206275696C6420257320FE
:10E600002573202A2A2A0A006F73006D61696E0043
:10E6100069646C65000000000080000045C60000D1
:10E620001BCA0000A1D4000000C2010000010300C9
:10E63000000000000090D003D4470120D4470120FF
:10E6400040DC000000000000000000007CDC000056
:10E650000000000000000000C4DC0000000000001A
:10E6600000000000D0DC00000000000000000000FE
:10E6700058DC0000000000000000000088DC000002
:10E68000000000000000000064DC0000A8DD0000C5
:10E6900018010120ACDC000030DE0000C44701207E
:10E6A00070DC000000000000000000004CDC0000F6
:10E6B0000000000000000000A0DC000004DE0000FC
:10E6C000F001012094DC000004DE000010020120B3
:10E6D000B8DC0000000000000000000078480120C5
:10E6E0007848012000000000010000008848012057
:10E6F0008848012000000000000000000F0000001A
:10E700009C4801209C4801200000000000000000FF
:04E710000F000000F6
:00000001FF
